:020000040000FA
:3C000000FFFF627515FFFFFFFFFFFFFFFFFFFFFFFFFFFFFFFFFFFFFFFFFFFFFFFFFFFFFFFFFFFFFFFFFFFFFFFFFFFFFFFFFFFFFFFFFFFFFFFFFFFFFFFFFFFFFF11
:3C003C00000000000000000000000000000000000008000000080008000000000000000000000000000000000000000000000000000000000000000000009EFED4
:3C0078000000000000000000000000000000000004800400048000800000040000000000000000000000040000000000000000000000000000000000000096FE24
:3C00B40000000000000000000000048000000000000000000000000004000000000000000000040004800000048000800400048000800480040004800000DAFE10
:3C00F0000000048004800480048000800480048014A8148814A804A004801488048004800480008004801488048004800480048004000080048004800000F8FEA6
:3C012C0000000480048004800480048004800480048804800488248004800480048004800480048024800480348024800480248004800488048004900000B6FE1F
:3C016800000004000480000000000480000000000480040004800080040004000000000000000400048004000480008004000480008004800400048000001AFEFF
:3C01A4000000008000000480048004800480048004800480048004800480048004800480048004800480048004800480048004800480048004800480000056FE67
:3C01E00000000080000004800480048004800480304030803040042034803080048004800480048004A0308024A004A034800CA8048034C00C880CA8000072FF52
:3C021C0000000000000000000000000000000000000000000000000000000000000000000000000000000000000000000000000000000000000000C40600ADFF30
:3C025800000000000000000000000000000000000000000000000000000000000000000000000000000000000000000000000000000000000000000002003CFE2E
:3C02940000000000000000000000000000000000000000000000000000000000000000000000000000000000000000000000000000000000000000800600F8FEB2
:3C02D00002000000000000000000000000000000000000000000000000000000000000000000000000000000000000000000000000000000000000801601C9FE92
:3C030C0002000000000000000000000000000000000000000000000000000000000000000000000000000000000000000000000000000000000000A4083021FEB8
:3C034800020000000000000000000000000000000000000000000000000000000000000000000000000000000000000000000000000000000000000000002FFF49
:3C03840000000000000000000000000000000000000000000000000000000000000000000000000000000000000000000000000000000000000000800500CBFEEF
:3C03C0000000000000000000000000000000000000000000000000000000000000000000000000000000000000000000000000000000008001000080000457FEA7
:3C03FC0000000000000000000000000000000000000000000000000000000000000000000000000000000084060000000000000000000000000000C2060074FE01
:3C043800000000000000000000000000000000000000000000000000000000000000000000000000000000000600000000000000000000000000000002003AFE48
:3C0474000000000000000000000000000000000000000000000000000000000000000000000000000000008004000000000000000000000000000080060074FED0
:3C04B000020000000000000000000000000000000000000000000000000000000000000000000000000000A014020000000000000000000000000080160155FE6E
:3C04EC0002000000000000000000000000000000000000000000000000000000000000000000000000000080100000000000000000000000000000A4000013FF8C
:3C052800000000000000000000000000000000000000000000000000000000000000000000000000000000000000000000000000000000000000000000001EFE7B
:3C0564000200000000000000000000000000000000000000000000000000000000000000000000000000008004000000000000000000000001000080040077FEDB
:3C05A00002000000000000000000000000000000000000000000000000000000000000000000000000000000020800000000000000000080000000000804E5FFA3
:3C05DC00000000000000000000000000000000000000000000000000000000000000000000000000000080C00E000000000000000000000000004080060067FF69
:3C061800000000000000000000000000000000000000000000000000000000000000000000000000000000000600000000000000000000000000000002003AFE66
:3C0654000000000000000000000000000000000000000000000000000000000000000000000000000000008002000000000000000000000000000080060072FEF2
:3C06900002000000000000000000000000000000000000000000000000000000000000000000000000000080220000000000000000000000000000A0160143FE92
:3C06CC0002000000000000000000000000000000000000000000000000000000000000000000000000000080100000000000000000000000000000A4005057FE17
:3C070800020000000000000000000000000000000000000000000000000000000000000000000000000000000000000000000000000000000000000000002FFF85
:3C0744000000000000000000000000000000000000000000000000000000000000000000000000000000008002000000000000000000000000000080040041FF33
:3C078000000000000000000000000000000000000000000000000000000000000000000000000000000000000408000000000000000000800100000088009BFE8F
:3C07BC0000000000000000000000000000000000000000000000000000000000000000A4160000A416A446C0060000000000000000000000000000A416002DFEF8
:3C07F800000000000000000000000000000000000000000000000000000000000000000006000000060002000600000000000000000000000000000006005AFE53
:3C08340000000000000000000000000000000000000000000000000000000000000000800000008000000480060000000000000000000000000000800000DCFEA4
:3C087000020000000000000000000000000000000000000000000000000000000000008020000080208008820E0400000000000000000000000000802000EFFF60
:3C08AC000200000000000000000000000000000000000000000000000000000000000084000080C00028088004000000000000000000000000000082001089FE7D
:3C08E800020000000000000000000000000000000000000000000000000000000000000002000000020000000200000000000000000000000000000002000DFFBE
:3C092400000000000000000000000000000000000000000000000000000000000000008002000080028004800600000000000000000000000000008002006DFF9B
:3C096000000000000000000000000000000000000000000000000000000000000000002016010000160142000E0100000000000000800100000000A0174113FE32
:3C099C00000000000000000000000000000000C10682468006A206C846C0020000000000000000A856C00288068806A80E8806A406880600008106C206001DFFCF
:3C09D800000000000000000000000000000000000600060006000600060002000000000000000000060002000600060006000600060006000000020006005EFE33
:3C0A1400000000000000000000000000000000800680068006800680028002000000000000000080008002800280028000800280008002000080048006001CFE5C
:3C0A50000200000000000000000000000000008036C036A036803680328032000000000000000080208032C032C0328080C0328030C08A0000A030803000E1FE4B
:3C0A8C00020000000000000000000000000040C010A848C010A8088010A81400000000000000008004A8148010801080048010880080000000A410A820002BFF3E
:3C0AC800020000000000000000000000000000000000000000000000000002000000000000000000020002000000000002000000020000000000000000000DFFDA
:3C0B0400000000000000000000000000000000800280028002800380028006000000000000000080048006800280028004800280028001000080068006003FFF43
:3C0B400000000000000000000000000000000000000840000088400004080204000000000000000032002200040804083200042816810801000006040020D7FFED
:3C0B7C00000000000000000000000000000000000000000000000000000000000000000000000000000080800E0000000000000000000000000000900E00EEFEA5
:3C0BB800000000000000000000000000000000000000000000000000000000000000000000000000000000000200000000000000000000000000000006007AFE81
:3C0BF400000000000000000000000000000000000000000000000000000000000000000000000000000000000000000000000000000000000000008000009EFEA9
:3C0C3000020000000000000000000000000000000000000000000000000000000000000000000000000000C0220000000000000000000000000000A0060227FFD6
:3C0C6C0002000000000000000000000000000000000000000000000000000000000000000000000000004040100000000000000000000000000000A80000D7FF3C
:3C0CA800020000000000000000000000000000000000000000000000000000000000000000000000000000000000000000000000000000000000000000003EFED2
:3C0CE4000000000000000000000000000000000000000000000000000000000000000000000000000000008000000000000000000000000000000080000007FFCE
:3C0D200000000000000000000000000000000000000000000000000000000000000000000000000000000000060800000000000000000000000000000600E7FF9D
:3C0D5C00000000000000000000000000000000000000000000000000000000000000000000000000000000900E0000000000000000000000000000C416002AFEBB
:3C0D9800000000000000000000000000000000000000000000000000000000000000000000000000000000000200000000000000000000000000000006007AFE9F
:3C0DD40000000000000000000000000000000000000000000000000000000000000000000000000000000000060000000000000000000000000000800600FEFE5B
:3C0E1000020000000000000000000000000000000000000000000000000000000000000000000000000000C000040000000000000000000000000080001027FE2B
:3C0E4C0002000000000000000000000000000000000000000000000000000000000000000000000000004040100000000000000000000000000000A80000D7FF5A
:3C0E8800000000000000000000000000000000000000000000000000000000000000000000000000000000000000000000000000000000000000000000001EFE12
:3C0EC4000200000000000000000000000000000000000000000000000000000000000000000000000000008004000000000000000000000000000080060045FFA2
:3C0F000002000000000000000000000000000000000000000000000000000000000000000000000000000000000800000000000000800180010000000000BFFFEB
:3C0F3C0000000000000000000000000000000000000000000000000000000000000000000000000000000084060000000000000000000000000000A816000EFF24
:3C0F7800000000000000000000000000000000000000000000000000000000000000000000000000000000000200000000000000000000000000000006007AFEBD
:3C0FB4000000000000000000000000000000000000000000000000000000000000000000000000000000000006000000000000000000000000000080000098FEE5
:3C0FF000020000000000000000000000000000000000000000000000000000000000000000000000000000A010040000000000000000000000000080200053FF1D
:3C102C0002000000000000000000000000000000000000000000000000000000000000000000000000004040100000000000000000000000000000800C0033FF38
:3C106800000000000000000000000000000000000000000000000000000000000000000000000000000000000000000000000000000000000000000002003CFE10
:3C10A4000200000000000000000000000000000000000000000000000000000000000000000000000000008004000000000000000000000000000080050067FEA0
:3C10E0000200000000000000000000000000000000000000000000000000000000000000008001800100000000080000000000000080010000000080021005FEB2
:3C111C0000000000000000000000000000000000000000000000000000000000000000000000009006900E9016000000000000000000000000004080060024FED5
:3C1158000000000000000000000000000000000000000000000000000000000000000000000000000200060006000000000000000000000000000000060038FE11
:3C119400000000000000000000000000000000000000000000000000000000000000000000000080068000800400000000000000000000000000008006009CFE75
:3C11D0000200000000000000000000000000000000000000000000000000000000000000000000C016C106C1040100000000000000000000000000A0081005FFC2
:3C120C000200000000000000000000000000000000000000000000000000000000000000000000A410A80080100000000000000000000000000000A80000F9FE19
:3C124800000000000000000000000000000000000000000000000000000000000000000000000000000000000000000000000000000000000000000000001EFE4E
:3C128400020000000000000000000000000000000000000000000000000000000000000000000080048000800400000001000000000000000000008006008DFE92
:3C12C0000200000000000000000000000000000000000000000000800100000000000000008001000002068003080080000000000000000000000000000059FF83
:3C12FC000000000000000000000000000000000000880E0000881600000000000000000000000000009006880688060000880688068800881688068806000EFE66
:3C13380000000000000000000000000000000000000006000000060000000080000000000000000000000200020002000000020006000600060006000600F4FED5
:3C137400000000000000000000000000000000000080000000800000000000000000000000000000000002800680060000800680048004800480048000001CFEFF
:3C13B0000200000000000000000000000000000000C0840000C0440000000000000000000000000000C092C016C1160100C016C134C016C104C134C016047DFF06
:3C13EC000200000000000000000000000000000000A8080000A80800000000000000000000000000002808A4108210000082108010A81080108010A800004FFFFD
:3C14280000800080008000800080008000800080008000800080008000800080008000800080008000800080008000800080008000800480008000800000DAFEAC
:3C1464000200000000000000000000000000000000000600000006000000000000000000000000000000000004000000000000000400000004000500000059FFD5
:3C14A000020000000000000000000000000000000000460000004680018001800080010000000000008045800121040400400404020800040288028807007BFE26
:3C14DC00000000000000000000000000000000000000000000000000000000000000000000000000000000000000000000000000000000000000000000001EFEB8
:3C151800000000000000000000000000000000200020002000200020002000000000002000000020002000200020002000200020002000200020002000001CFE3D
:3C155400000000000000000000000000000000000000000000000000000000000000000000000000000000000000000000000000000000000000000000001EFE3F
:3C159000000000000000000000000000000000000000000000000000000000000000000000000000000000000000000000000000000000000000000000001EFE03
:3C15CC00000000000000000000000000000000000000000000000000000000000000000002000000000000000000000000000000000000000000000000201EFEA5
:3C160800000000000000000000000000000000000000000000000000000000000000000000000000000000000000000000000000000000000000000000001EFE8A
:3C164400000000000000000000000000000000000000000000000000000000000000000000000000000000000000000000000000000000000000000000001EFE4E
:3C168000000000000000000000000000000000000000000000000000000000000000000000000000000000010400000000080000000000000000000000008AFE99
:3C16BC00000000000000000000000000000000000000000000000000000000000000000000000000000010002000000000000020000020000000020001000EFE73
:3C16F800000000000000000000000000000000000000000000000100000000000000024000000400002200000040000000000000000000000020000000004EFFA0
:3C17340000000000000000000000000000000000004000400040004000000040000000000000000000000040000000004000000000800400000000000000DAFE5D
:3C1770000000000000000000000000000000000000080000000000000000000000000000000000000000000000000000000000000000010000000000000096FF9F
:3C17AC00000000000000000000000000000000000000000000000000000000000000000000000000000000000000000000000000000000000000000000001EFEE5
:3C17E800000000000000000000000000000000000000000000000000000000000000000080002000800020008400800002008000800080008000000080001AFEE7
:3C182400000000000000000000000000000000000000200000000000000000000000002000000020000004A000000020000000200000402000000020040090FE32
:3C18600000000000000000000000000000000000000000000000000006000400040000000000000000002000001000000000000000000000000000022018ACFE2A
:3C189C00000000000000000000000000000000000000000000020000000000000000000000000000000000000000000000000000000000040000000000007EFE8E
:3C18D80000000000000000000000000000000000000000000000000000000020000000000000000000000000000000000000000000000008000000044000BCFEAE
:3C191400000000000000000000000000000000000000000000000000000000000000000000000000000000000000000000000000000000000000000000001EFE7B
:3C195000000000000000000000000000000000000000000000000000000000000000000000000000000000404000000000000000000000000000000000001AFEC3
:3C198C00000000000000000000000000000000010000000000000000000000000000000000000000000000001000000000000000000000000000000000001EFEF2
:3C19C800000000000000000000000000000000000000080000000000000000000000000000000000000000008000000000000000000000000000000000001EFE3F
:3C1A0400000000000000000000000000000000000000000000000000000000000000000000000000000000000000000000000000000000000000000000001EFE8A
:3C1A4000000000000000000000000000000000000000000000000000000000000000000000000000000000000000000000000000000010000001000000000EFE4D
:3C1A7C000000000000000000000000000000000000000000000000000000000000000000000000000000000000080000000000000000004000001040000092FF05
:3C1AB8000000000000000000000000000000040000000400000004000400000000000000000008000C00040080020000000000000000000020000000000050FEDA
:3C1AF400000000000000000000000000000000000000000000000000000000000000000000000000000000000000000000000000000000000000000000001EFE9A
:3C1B3000000000000000000000000000000000000000000000000000000000000000000000000000000000000000000000000000000000000000000000001EFE5D
:3C1B6C00000000000000000000000000000000000000000000000000000000000000000000000000000000000000000000000000000000000000000000001EFE21
:3C1BA800000000000000000000000000000000000000000000000000010000000000000000000000000000000000000000000000000020000000000000000CFED6
:3C1BE400000000000000000000000000000000000000000000000200000000000000000000000000000400080000000000000000000000000000000200009AFE1D
:3C1C200000000000000000000000000000000000008000000080000000800000000000000000009000800000008000800000008000800000008000800804C6FF27
:3C1C5C00000000000000000000000000000000000000000000000000000000000000000000000000000000000000000000000000000000000000000000001EFE30
:3C1C9800000000000000000000000000000000000000000000000000000000000000000000000000000000000000000000000000000000000000000000001EFEF4
:3C1CD400000000000000000000000000000000000000000000000000000000000000000000000000000000000000000000000000000000000000000000001EFEB8
:3C1D10000000000000000000000000000000000000000000000000000000000000000000000000000000000000000000000000000000000000000008000106FE8A
:3C1D4C00000000000000000000000000000000000000000000000000000000000000000000000000000000000000000000000000000000000000000000000FFF4D
:3C1D8800000000000000000000000000000000000000000000000000000000000000000000000000000000000000000000000000000000000000000000001EFE03
:3C1DC400000000000000000000000000000000000000000000000000000000000000000000000000000000000000000000000000000000000000000000001EFEC7
:3C1E0000020000000000000000000000000000000000000000000000000000000000000000000000000000000000000000000000000000000000000000003EFE68
:3C1E3C00020000000000000000000000000000000000000000000000000000000000000000000000000000000000000000000000000000000000000000002FFF3A
:3C1E7800000000000000000000000000000000000000000000000000000000000000000000000000000000000000000000000000000000000000000000000FFF20
:3C1EB400020000000000000000000000000000000000000000000000000000000000000000000000000000000000000000000000000000000000000000003EFEB4
:3C1EF000020000000000000000000000000000000000000000000000000000000000000000000000000000000000000000000000000000000000000000003EFE78
:3C1F2C00020000000000000000000000000000000000000000000000000000000000000000000000000000000000000000000000000000000000000000003EFE3B
:3C1F6800000000000000000000000000000000000000000000000000000000000000000000000000000000000000000000000000000000000000000000001EFE21
:3C1FA400000000000000000000000000000000000000000000000000000000000000000000000000000000000000000000000000000000000000000000001EFEE5
:3C1FE000020000000000000000000000000000000000000000000000000000000000000000000000000000000000000000000000000000000000000000002FFF95
:3C201C00020000000000000000000000000000000000000000000000000000000000000000000000000000000000000000000000000000000000000000002FFF58
:3C205800020000000000000000000000000000000000000000000000000000000000000000000000000000000000000000000000000000000000000000002FFF1C
:3C209400020000000000000000000000000000000000000000000000000000000000000000000000000000000000000000000000000000000000000000003EFED2
:3C20D000020000000000000000000000000000000000000000000000000000000000000000000000000000000000000000000000000000000000000000003EFE96
:3C210C00000000000000000000000000000000000000000000000000000000000000000000000000000000000000000000000000000000000000000000001EFE7B
:3C214800000000000000000000000000000000000000000000000000000000000000000000000000000000000000000000000000000000000000000000001EFE3F
:3C218400000000000000000000000000000000000000000000000000000000000000000000000000000000000000000000000000000000000000000000001EFE03
:3C21C000020000000000000000000000000000000000000000000000000000000000000000000000000000000000000000000000000000000000000000002FFFB3
:3C21FC00020000000000000000000000000000000000000000000000000000000000000000000000000000000000000000000000000000000000000000002FFF77
:3C223800000000000000000000000000000000000000000000000000000000000000000000000000000000000000000000000000000000000000000000001EFE4E
:3C227400020000000000000000000000000000000000000000000000000000000000000000000000000000000000000000000000000000000000000000002FFFFE
:3C22B000020000000000000000000000000000000000000000000000000000000000000000000000000000000000000000000000000000000000000000002FFFC2
:3C22EC00020000000000000000000000000000000000000000000000000000000000000000000000000000000000000000000000000000000000000000003EFE78
:3C232800000000000000000000000000000000000000000000000000000000000000000000000000000000000000000000000000000000000000000000001EFE5D
:3C236400000000000000000000000000000000000000000000000000000000000000000000000000000000000000000000000000000000000000000000001EFE21
:3C23A000020000000000000000000000000000000000000000000000000000000000000000000000000000000000000000000000000000000000000000002FFFD1
:3C23DC00020000000000000000000000000000000000000000000000000000000000000000000000000000000000000000000000000000000000000000002FFF95
:3C241800020000000000000000000000000000000000000000000000000000000000000000000000000000000000000000000000000000000000000000003EFE4A
:3C245400020000000000000000000000000000000000000000000000000000000000000000000000000000000000000000000000000000000000000000002FFF1C
:3C249000020000000000000000000000000000000000000000000000000000000000000000000000000000000000000000000000000000000000000000002FFFE0
:3C24CC00000000000000000000000000000000000000000000000000000000000000000000000000000000000000000000000000000000000000000000000FFFC6
:3C250800000000000000000000000000000000000000000000000000000000000000000000000000000000000000000000000000000000000000000000001EFE7B
:3C254400000000000000000000000000000000000000000000000000000000000000000000000000000000000000000000000000000000000000000000001EFE3F
:3C258000020000000000000000000000000000000000000000000000000000000000000000000000000000000000000000000000000000000000000000003EFEE1
:3C25BC00020000000000000000000000000000000000000000000000000000000000000000000000000000000000000000000000000000000000000000002FFFB3
:3C25F800000000000000000000000000000000000000000000000000000000000000000000000000000000000000000000000000000000000000000000000FFF99
:3C263400020000000000000000000000000000000000000000000000000000000000000000000000000000000000000000000000000000000000000000003EFE2C
:3C267000020000000000000000000000000000000000000000000000000000000000000000000000000000000000000000000000000000000000000000003EFEF0
:3C26AC00000000000000000000000000000000000000000000000000000000000000000000000000000000000000000000000000000000000000000000001EFED6
:3C26E800000000000000000000000000000000000000000000000000000000000000000000000000000000000000000000000000000000000000000000001EFE9A
:3C272400000000000000000000000000000000000000000000000000000000000000000000000000000000000000000000000000000000000000000000001EFE5D
:3C276000020000000000000000000000000000000000000000000000000000000000000000000000000000000000000000000000000000000000000000002FFF0D
:3C279C00020000000000000000000000000000000000000000000000000000000000000000000000000000000000000000000000000000000000000000002FFFD1
:3C27D800000000000000000000000000000000000000000000000000000000000000000000000000000000000000000000000000000000000000000000001EFEA9
:3C281400020000000000000000000000000000000000000000000000000000000000000000000000000000000000000000000000000000000000000000002FFF58
:3C285000020000000000000000000000000000000000000000000000000000000000000000000000000000000000000000000000000000000000000000002FFF1C
:3C288C00000000000000000000000000000000000000000000000000000000000000000000000000000000000000000000000000000000000000000000000FFF02
:3C28C800000000000000000000000000000000000000000000000000000000000000000000000000000000000000000000000000000000000000000000001EFEB8
:3C290400000000000000000000000000000000000000000000000000000000000000000000000000000000000000000000000000000000000000000000001EFE7B
:3C294000020000000000000000000000000000000000000000000000000000000000000000000000000000000000000000000000000000000000000000003EFE1D
:3C297C00020000000000000000000000000000000000000000000000000000000000000000000000000000000000000000000000000000000000000000002FFFEF
:3C29B800000000000000000000000000000000000000000000000000000000000000000000000000000000000000000000000000000000000000000000000FFFD5
:3C29F400020000000000000000000000000000000000000000000000000000000000000000000000000000000000000000000000000000000000000000003EFE69
:3C2A3000020000000000000000000000000000000000000000000000000000000000000000000000000000000000000000000000000000000000000000003EFE2C
:3C2A6C00000000000000000000000000000000000000000000000000000000000000000000000000000000000000000000000000000000000000000000000FFF20
:3C2AA800000000000000000000000000000000000000000000000000000000000000000000000000000000000000000000000000000000000000000000001EFED6
:3C2AE400000000000000000000000000000000000000000000000000000000000000000000000000000000000000000000000000000000000000000000001EFE9A
:3C2B2000020000000000000000000000000000000000000000000000000000000000000000000000000000000000000000000000000000000000000000003EFE3B
:3C2B5C00020000000000000000000000000000000000000000000000000000000000000000000000000000000000000000000000000000000000000000002FFF0D
:3C2B9800000000000000000000000000000000000000000000000000000000000000000000000000000000000000000000000000000000000000000000000FFFF3
:3C2BD400020000000000000000000000000000000000000000000000000000000000000000000000000000000000000000000000000000000000000000003EFE87
:3C2C1000020000000000000000000000000000000000000000000000000000000000000000000000000000000000000000000000000000000000000000003EFE4A
:3C2C4C00000000000000000000000000000000000000000000000000000000000000000000000000000000000000000000000000000000000000000000001EFE30
:3C2C8800000000000000000000000000000000000000000000000000000000000000000000000000000000000000000000000000000000000000000000001EFEF4
:3C2CC400000000000000000000000000000000000000000000000000000000000000000000000000000000000000000000000000000000000000000000001EFEB8
:3C2D0000020000000000000000000000000000000000000000000000000000000000000000000000000000000000000000000000000000000000000000002FFF67
:3C2D3C00020000000000000000000000000000000000000000000000000000000000000000000000000000000000000000000000000000000000000000002FFF2B
:3C2D7800020000000000000000000000000000000000000000000000000000000000000000000000000000000000000000000000000000000000000000003EFEE1
:3C2DB400000000000000000000000000000000000000000000000000000000000000000000000000000000000000000000000000000000000000000000000FFFD5
:3C2DF000000000000000000000000000000000000000000000000000000000000000000000000000000000000000000000000000000000000000000000000FFF99
:3C2E2C00000000000000000000000000000000000000000000000000000000000000000000000000000000000000000000000000000000000000000000000FFF5C
:3C2E6800000000000000000000000000000000000000000000000000000000000000000000000000000000000000000000000000000000000000000000001EFE12
:3C2EA400000000000000000000000000000000000000000000000000000000000000000000000000000000000000000000000000000000000000000000001EFED6
:3C2EE000020000000000000000000000000000000000000000000000000000000000000000000000000000000000000000000000000000000000000000003EFE78
:3C2F1C00020000000000000000000000000000000000000000000000000000000000000000000000000000000000000000000000000000000000000000002FFF49
:3C2F5800008000800080008000800080008000800080008000800080008000800080008000800080008000800080008000800080008000800080008000008FFFAF
:3C2F9400020000000000000000000000000000000000000000000000000000000000000000000000000000000000000000000000000000000000000000003EFEC3
:3C2FD000020000000000000000000000000000000000000000000000000000000000000000000000000000000000000000000000000000000000000000003EFE87
:3C300C00000000000000000000000000000000000000000000000000000000000000000000000000000000000000000000000000000000000000000000001EFE6C
:3C304800000000000000000000000000000000000000000000000000000000000000000000000000000000000000000000000000000000000000000000001EFE30
:3C308400000000000000000000000000000000000000000000000000000000000000000000000000000000000000000000000000000000000000000000001EFEF4
:3C30C000000000000000000000000000000000000000000000000000000000000000000000000000000000000000000000000000000000000000000000001EFEB8
:3C30FC00000000000000000000000000000000000000000000000000000000000000000000000000000000000000000000000000000000000000000000001EFE7C
:3C313800000000000000000000000000000000000000000000000000000000000000000000000000000000000000000000000000000000000000000000001EFE3F
:3C317400000000000000000000000000000000000000000000000000000000000000000000000000000000000000000000000000000000000000000000001EFE03
:3C31B000000000000000000000000000000000000000000000000000000000000000000000000000000000000000000000000000000000000000000000001EFEC7
:3C31EC00000000000000000000000000000000000000000000000000000000000000000000000000000000000000000000000000000000000000000000001EFE8B
:3C322800000000000000000000000000000000000000000000000000000000000000000000000000000000000000000000000000000000000000000000001EFE4E
:3C326400000000000000000000000000000000000000000000000000000000000000000000000000000000000000000000000000000000000000000000001EFE12
:3C32A000000000000000000000000000000000000000000000000000000000000000000000000000000000000000000000000000000000000000000000001EFED6
:3C32DC00000000000000000000000000000000000000000000000000000000000000000000000000000000000000000000000000000000000000000000001EFE9A
:3C331800000000000000000000000000000000000000000000000000000000000000000000000000000000000000000000000000000000000000000000001EFE5D
:3C335400000000000000000000000000000000000000000000000000000000000000000000000000000000000000000000000000000000000000000000001EFE21
:3C339000000000000000000000000000000000000000000000000000000000000000000000000000000000000000000000000000000000000000000000001EFEE5
:3C33CC00000000000000000000000000000000000000000000000000000000000000000000000000000000000000000000000000000000000000000000001EFEA9
:3C340800000000000000000000000000000000000000000000000000000000000000000000000000000000000000000000000000000000000000000000001EFE6C
:3C344400000000000000000000000000000000000000000000000000000000000000000000000000000000000000000000000000000000000000000000001EFE30
:3C348000000000000000000000000000000000000000000000000000000000000000000000000000000000000000000000000000000000000000000000001EFEF4
:3C34BC00000000000000000000000000000000000000000000000000000000000000000000000000000000000000000000000000000000000000000000001EFEB8
:3C34F800000000000000000000000000000000000000000000000000000000000000000000000000000000000000000000000000000000000000000000001EFE7C
:3C353400000000000000000000000000000000000000000000000000000000000000000000000000000000000000000000000000000000000000000000001EFE3F
:3C357000000000000000000000000000000000000000000000000000000000000000000000000000000000000000000000000000000000000000000000001EFE03
:3C35AC00000000000000000000000000000000000000000000000000000000000000000000000000000000000000000000000000000000000000000000001EFEC7
:3C35E800000000000000000000000000000000000000000000000000000000000000000000000000000000000000000000000000000000000000000000001EFE8B
:3C362400000000000000000000000000000000000000000000000000000000000000000000000000000000000000000000000000000000000000000000001EFE4E
:3C366000000000000000000000000000000000000000000000000000000000000000000000000000000000000000000000000000000000000000000000001EFE12
:3C369C00000000000000000000000000000000000000000000000000000000000000000000000000000000000000000000000000000000000000000000001EFED6
:3C36D800000000000000000000000000000000000000000000000000000000000000000000000000000000000000000000000000000000000000000000001EFE9A
:3C371400000000000000000000000000000000000000000000000000000000000000000000000000000000000000000000000000000000000000000000001EFE5D
:3C375000000000000000000000000000000000000000000000000000000000000000000000000000000000000000000000000000000000000000000000001EFE21
:3C378C00000000000000000000000000000000000000000000000000000000000000000000000000000000000000000000000000000000000000000000001EFEE5
:3C37C800000000000000000000000000000000000000000000000000000000000000000000000000000000000000000000000000000000000000000000001EFEA9
:3C380400000000000000000000000000000000000000000000000000000000000000000000000000000000000000000000000000000000000000000000001EFE6C
:3C384000000000000000000000000000000000000000000000000000000000000000000000000000000000000000000000000000000000000000000000001EFE30
:3C387C00000000000000000000000000000000000000000000000000000000000000000000000000000000000000000000000000000000000000000000001EFEF4
:3C38B800000000000000000000000000000000000000000000000000000000000000000000000000000000000000000000000000000000000000000000001EFEB8
:3C38F400000000000000000000000000000000000000000000000000000000000000000000000000000000000000000000000000000000000000000000001EFE7C
:3C393000020000000000000000000000000000000000000000000000000000000000000000000000000000000000000000000000000000000000000000002FFF2B
:3C396C00020000000000000000000000000000000000000000000000000000000000000000000000000000000000000000000000000000000000000000002FFFEF
:3C39A800000000000000000000000000000000000000000000000000000000000000000000000000000000000000000000000000000000000000000000001EFEC7
:3C39E400020000000000000000000000000000000000000000000000000000000000000000000000000000000000000000000000000000000000000000002FFF77
:3C3A2000020000000000000000000000000000000000000000000000000000000000000000000000000000000000000000000000000000000000000000002FFF3A
:3C3A5C00000000000000000000000000000000000000000000000000000000000000000000000000000000000000000000000000000000000000000000001EFE12
:3C3A9800000000000000000000000000000000000000000000000000000000000000000000000000000000000000000000000000000000000000000000001EFED6
:3C3AD400000000000000000000000000000000000000000000000000000000000000000000000000000000000000000000000000000000000000000000001EFE9A
:3C3B1000020000000000000000000000000000000000000000000000000000000000000000000000000000000000000000000000000000000000000000002FFF49
:3C3B4C00020000000000000000000000000000000000000000000000000000000000000000000000000000000000000000000000000000000000000000002FFF0D
:3C3B8800020000000000000000000000000000000000000000000000000000000000000000000000000000000000000000000000000000000000000000003EFEC3
:3C3BC400000000000000000000000000000000000000000000000000000000000000000000000000000000000000000000000000000000000000000000000FFFB7
:3C3C0000000000000000000000000000000000000000000000000000000000000000000000000000000000000000000000000000000000000000000000000FFF7A
:3C3C3C00000000000000000000000000000000000000000000000000000000000000000000000000000000000000000000000000000000000000000000000FFF3E
:3C3C7800000000000000000000000000000000000000000000000000000000000000000000000000000000000000000000000000000000000000000000001EFEF4
:3C3CB400000000000000000000000000000000000000000000000000000000000000000000000000000000000000000000000000000000000000000000001EFEB8
:3C3CF000020000000000000000000000000000000000000000000000000000000000000000000000000000000000000000000000000000000000000000002FFF68
:3C3D2C00020000000000000000000000000000000000000000000000000000000000000000000000000000000000000000000000000000000000000000002FFF2B
:3C3D6800020000000000000000000000000000000000000000000000000000000000000000000000000000000000000000000000000000000000000000002FFFEF
:3C3DA400000000000000000000000000000000000000000000000000000000000000000000000000000000000000000000000000000000000000000000000FFFD5
:3C3DE000000000000000000000000000000000000000000000000000000000000000000000000000000000000000000000000000000000000000000000000FFF99
:3C3E1C00000000000000000000000000000000000000000000000000000000000000000000000000000000000000000000000000000000000000000000000FFF5C
:3C3E5800000000000000000000000000000000000000000000000000000000000000000000000000000000000000000000000000000000000000000000001EFE12
:3C3E9400000000000000000000000000000000000000000000000000000000000000000000000000000000000000000000000000000000000000000000001EFED6
:3C3ED000020000000000000000000000000000000000000000000000000000000000000000000000000000000000000000000000000000000000000000002FFF86
:3C3F0C00020000000000000000000000000000000000000000000000000000000000000000000000000000000000000000000000000000000000000000002FFF49
:3C3F4800020000000000000000000000000000000000000000000000000000000000000000000000000000000000000000000000000000000000000000002FFF0D
:3C3F8400000000000000000000000000000000000000000000000000000000000000000000000000000000000000000000000000000000000000000000000FFFF3
:3C3FC000000000000000000000000000000000000000000000000000000000000000000000000000000000000000000000000000000000000000000000000FFFB7
:3C3FFC00000000000000000000000000000000000000000000000000000000000000000000000000000000000000000000000000000000000000000000000FFF7B
:3C403800000000000000000000000000000000000000000000000000000000000000000000000000000000000000000000000000000000000000000000001EFE30
:3C407400000000000000000000000000000000000000000000000000000000000000000000000000000000000000000000000000000000000000000000001EFEF4
:3C40B000020000000000000000000000000000000000000000000000000000000000000000000000000000000000000000000000000000000000000000002FFFA4
:3C40EC00020000000000000000000000000000000000000000000000000000000000000000000000000000000000000000000000000000000000000000002FFF68
:3C412800020000000000000000000000000000000000000000000000000000000000000000000000000000000000000000000000000000000000000000002FFF2B
:3C416400000000000000000000000000000000000000000000000000000000000000000000000000000000000000000000000000000000000000000000000FFF11
:3C41A000000000000000000000000000000000000000000000000000000000000000000000000000000000000000000000000000000000000000000000000FFFD5
:3C41DC00000000000000000000000000000000000000000000000000000000000000000000000000000000000000000000000000000000000000000000000FFF99
:3C421800000000000000000000000000000000000000000000000000000000000000000000000000000000000000000000000000000000000000000000001EFE4E
:3C425400000000000000000000000000000000000000000000000000000000000000000000000000000000000000000000000000000000000000000000001EFE12
:3C429000020000000000000000000000000000000000000000000000000000000000000000000000000000000000000000000000000000000000000000002FFFC2
:3C42CC00020000000000000000000000000000000000000000000000000000000000000000000000000000000000000000000000000000000000000000002FFF86
:3C430800020000000000000000000000000000000000000000000000000000000000000000000000000000000000000000000000000000000000000000002FFF49
:3C434400000000000000000000000000000000000000000000000000000000000000000000000000000000000000000000000000000000000000000000000FFF2F
:3C438000000000000000000000000000000000000000000000000000000000000000000000000000000000000000000000000000000000000000000000000FFFF3
:3C43BC00000000000000000000000000000000000000000000000000000000000000000000000000000000000000000000000000000000000000000000001EFEA9
:3C43F800000000000000000000000000000000000000000000000000000000000000000000000000000000000000000000000000000000000000000000001EFE6D
:3C443400000000000000000000000000000000000000000000000000000000000000000000000000000000000000000000000000000000000000000000001EFE30
:3C447000020000000000000000000000000000000000000000000000000000000000000000000000000000000000000000000000000000000000000000002FFFE0
:3C44AC00020000000000000000000000000000000000000000000000000000000000000000000000000000000000000000000000000000000000000000002FFFA4
:3C44E800000000000000000000000000000000000000000000000000000000000000000000000000000000000000000000000000000000000000000000001EFE7C
:3C452400020000000000000000000000000000000000000000000000000000000000000000000000000000000000000000000000000000000000000000002FFF2B
:3C456000020000000000000000000000000000000000000000000000000000000000000000000000000000000000000000000000000000000000000000002FFFEF
:3C459C00000000000000000000000000000000000000000000000000000000000000000000000000000000000000000000000000000000000000000000000FFFD5
:3C45D800000000000000000000000000000000000000000000000000000000000000000000000000000000000000000000000000000000000000000000001EFE8B
:3C461400000000000000000000000000000000000000000000000000000000000000000000000000000000000000000000000000000000000000000000001EFE4E
:3C465000020000000000000000000000000000000000000000000000000000000000000000000000000000000000000000000000000000000000000000003EFEF0
:3C468C00020000000000000000000000000000000000000000000000000000000000000000000000000000000000000000000000000000000000000000002FFFC2
:3C46C800020000000000000000000000000000000000000000000000000000000000000000000000000000000000000000000000000000000000000000002FFF86
:3C470400000000000000000000000000000000000000000000000000000000000000000000000000000000000000000000000000000000000000000000001EFE5D
:3C474000000000000000000000000000000000000000000000000000000000000000000000000000000000000000000000000000000000000000000000001EFE21
:3C477C00000000000000000000000000000000000000000000000000000000000000000000000000000000000000000000000000000000000000000000000FFFF3
:3C47B800000000000000000000000000000000000000000000000000000000000000000000000000000000000000000000000000000000000000000000001EFEA9
:3C47F400000000000000000000000000000000000000000000000000000000000000000000000000000000000000000000000000000000000000000000001EFE6D
:3C483000020000000000000000000000000000000000000000000000000000000000000000000000000000000000000000000000000000000000000000003EFE0E
:3C486C00020000000000000000000000000000000000000000000000000000000000000000000000000000000000000000000000000000000000000000002FFFE0
:3C48A800020000000000000000000000000000000000000000000000000000000000000000000000000000000000000000000000000000000000000000002FFFA4
:3C48E400000000000000000000000000000000000000000000000000000000000000000000000000000000000000000000000000000000000000000000000FFF8A
:3C492000000000000000000000000000000000000000000000000000000000000000000000000000000000000000000000000000000000000000000000000FFF4D
:3C495C00020000000000000000000000000000000000000000000000000000000000000000000000000000000000000000000000000000000000000000002FFFEF
:3C499800000000000000000000000000000000000000000000000000000000000000000000000000000000000000000000000000000000000000000000001EFEC7
:3C49D400000000000000000000000000000000000000000000000000000000000000000000000000000000000000000000000000000000000000000000001EFE8B
:3C4A1000000000000000000000000000000000000000000000000000000000000000000000000000000000000000000000000000000000000000000000001EFE4E
:3C4A4C00000000000000000000000000000000000000000000000000000000000000000000000000000000000000000000000000000000000000000000001EFE12
:3C4A8800008000800080008000800080008000800080008000800080008000800080008000800080008000800080008000800080008000800080008000009EFE56
:3C4AC400000000000000000000000000000000000000000000000000000000000000000000000000000000000000000000000000000000000000000000001EFE9A
:3C4B0000000000000000000000000000000000000000000000000000000000000000000000000000000000000000000000000000000000000000000000001EFE5D
:3C4B3C00000000000000000000000000000000000000000000000000000000000000000000000000000000000000000000000000000000000000000000001EFE21
:3C4B7800000000000000000000000000000000000000000000000000000000000000000000000000000000000000000000000000000000000000000000001EFEE5
:3C4BB400000000000000000000000000000000000000000000000000000000000000000000000000000000000000000000000000000000000000000000001EFEA9
:3C4BF000000000000000000000000000000000000000000000000000000000000000000000000000000000000000000000000000000000000000000000001EFE6D
:3C4C2C00000000000000000000000000000000000000000000000000000000000000000000000000000000000000000000000000000000000000000000001EFE30
:3C4C6800000000000000000000000000000000000000000000000000000000000000000000000000000000000000000000000000000000000000000000001EFEF4
:3C4CA400000000000000000000000000000000000000000000000000000000000000000000000000000000000000000000000000000000000000000000001EFEB8
:3C4CE000000000000000000000000000000000000000000000000000000000000000000000000000000000000000000000000000000000000000000000001EFE7C
:3C4D1C00000000000000000000000000000000000000000000000000000000000000000000000000000000000000000000000000000000000000000000001EFE3F
:3C4D5800000000000000000000000000000000000000000000000000000000000000000000000000000000000000000000000000000000000000000000001EFE03
:3C4D9400000000000000000000000000000000000000000000000000000000000000000000000000000000000000000000000000000000000000000000001EFEC7
:3C4DD000000000000000000000000000000000000000000000000000000000000000000000000000000000000000000000000000000000000000000000001EFE8B
:3C4E0C00000000000000000000000000000000000000000000000000000000000000000000000000000000000000000000000000000000000000000000001EFE4E
:3C4E4800000000000000000000000000000000000000000000000000000000000000000000000000000000000000000000000000000000000000000000001EFE12
:3C4E8400000000000000000000000000000000000000000000000000000000000000000000000000000000000000000000000000000000000000000000001EFED6
:3C4EC000000000000000000000000000000000000000000000000000000000000000000000000000000000000000000000000000000000000000000000001EFE9A
:3C4EFC00000000000000000000000000000000000000000000000000000000000000000000000000000000000000000000000000000000000000000000001EFE5E
:3C4F3800000000000000000000000000000000000000000000000000000000000000000000000000000000000000000000000000000000000000000000001EFE21
:3C4F7400000000000000000000000000000000000000000000000000000000000000000000000000000000000000000000000000000000000000000000001EFEE5
:3C4FB000000000000000000000000000000000000000000000000000000000000000000000000000000000000000000000000000000000000000000000001EFEA9
:3C4FEC00000000000000000000000000000000000000000000000000000000000000000000000000000000000000000000000000000000000000000000001EFE6D
:3C502800000000000000000000000000000000000000000000000000000000000000000000000000000000000000000000000000000000000000000000001EFE30
:3C506400000000000000000000000000000000000000000000000000000000000000000000000000000000000000000000000000000000000000000000001EFEF4
:3C50A000000000000000000000000000000000000000000000000000000000000000000000000000000000000000000000000000000000000000000000001EFEB8
:3C50DC00000000000000000000000000000000000000000000000000000000000000000000000000000000000000000000000000000000000000000000001EFE7C
:3C511800000000000000000000000000000000000000000000000000000000000000000000000000000000000000000000000000000000000000000000001EFE3F
:3C515400000000000000000000000000000000000000000000000000000000000000000000000000000000000000000000000000000000000000000000001EFE03
:3C519000000000000000000000000000000000000000000000000000000000000000000000000000000000000000000000000000000000000000000000001EFEC7
:3C51CC00000000000000000000000000000000000000000000000000000000000000000000000000000000000000000000000000000000000000000000001EFE8B
:3C520800000000000000000000000000000000000000000000000000000000000000000000000000000000000000000000000000000000000000000000001EFE4E
:3C524400000000000000000000000000000000000000000000000000000000000000000000000000000000000000000000000000000000000000000000001EFE12
:3C528000000000000000000000000000000000000000000000000000000000000000000000000000000000000000000000000000000000000000000000001EFED6
:3C52BC00000000000000000000000000000000000000000000000000000000000000000000000000000000000000000000000000000000000000000000001EFE9A
:3C52F800000000000000000000000000000000000000000000000000000000000000000000000000000000000000000000000000000000000000000000001EFE5E
:3C533400000000000000000000000000000000000000000000000000000000000000000000000000000000000000000000000000000000000000000000001EFE21
:3C537000000000000000000000000000000000000000000000000000000000000000000000000000000000000000000000000000000000000000000000001EFEE5
:3C53AC00000000000000000000000000000000000000000000000000000000000000000000000000000000000000000000000000000000000000000000000FFFB7
:3C53E800000000000000000000000000000000000000000000000000000000000000000000000000000000000000000000000000000000000000000000001EFE6D
:3C542400000000000000000000000000000000000000000000000000000000000000000000000000000000000000000000000000000000000000000000001EFE30
:3C546000020000000000000000000000000000000000000000000000000000000000000000000000000000000000000000000000000000000000000000003EFED2
:3C549C00020000000000000000000000000000000000000000000000000000000000000000000000000000000000000000000000000000000000000000002FFFA4
:3C54D800000000000000000000000000000000000000000000000000000000000000000000000000000000000000000000000000000000000000000000000FFF8A
:3C551400020000000000000000000000000000000000000000000000000000000000000000000000000000000000000000000000000000000000000000002FFF2B
:3C555000020000000000000000000000000000000000000000000000000000000000000000000000000000000000000000000000000000000000000000002FFFEF
:3C558C00020000000000000000000000000000000000000000000000000000000000000000000000000000000000000000000000000000000000000000002FFFB3
:3C55C800000000000000000000000000000000000000000000000000000000000000000000000000000000000000000000000000000000000000000000001EFE8B
:3C560400000000000000000000000000000000000000000000000000000000000000000000000000000000000000000000000000000000000000000000001EFE4E
:3C564000020000000000000000000000000000000000000000000000000000000000000000000000000000000000000000000000000000000000000000003EFEF0
:3C567C00020000000000000000000000000000000000000000000000000000000000000000000000000000000000000000000000000000000000000000002FFFC2
:3C56B800020000000000000000000000000000000000000000000000000000000000000000000000000000000000000000000000000000000000000000002FFF86
:3C56F400020000000000000000000000000000000000000000000000000000000000000000000000000000000000000000000000000000000000000000003EFE3C
:3C573000020000000000000000000000000000000000000000000000000000000000000000000000000000000000000000000000000000000000000000003EFEFF
:3C576C00000000000000000000000000000000000000000000000000000000000000000000000000000000000000000000000000000000000000000000001EFEE5
:3C57A800000000000000000000000000000000000000000000000000000000000000000000000000000000000000000000000000000000000000000000001EFEA9
:3C57E400000000000000000000000000000000000000000000000000000000000000000000000000000000000000000000000000000000000000000000001EFE6D
:3C582000020000000000000000000000000000000000000000000000000000000000000000000000000000000000000000000000000000000000000000002FFF1C
:3C585C00020000000000000000000000000000000000000000000000000000000000000000000000000000000000000000000000000000000000000000002FFFE0
:3C589800000000000000000000000000000000000000000000000000000000000000000000000000000000000000000000000000000000000000000000001EFEB8
:3C58D400020000000000000000000000000000000000000000000000000000000000000000000000000000000000000000000000000000000000000000002FFF68
:3C591000020000000000000000000000000000000000000000000000000000000000000000000000000000000000000000000000000000000000000000002FFF2B
:3C594C0002000000000000000000000000000000000000000000000000000000000000000000000000000000000000000000000000841600000000000000DDFEA8
:3C5988000000000000000000000000000000000000000000000000000000000000000000000000000000000000000000000000000000060000000000000078FE67
:3C59C40000000000000000000000000000000000000000000000000000000000000000000000000000000000000000000000000000800600000000000000F8FE2B
:3C5A000002000000000000000000000000000000000000000000000000000000000000000000000000000000000000000000000000C02000000000000000FCFE8E
:3C5A3C0002000000000000000000000000000000000000000000000000000000000000000000000000000000000000000000000040800000000000000000EBFF82
:3C5A7800020000000000000000000000000000000000000000000000000000000000000000000000000000000000000000000000000000000000000000002FFFC2
:3C5AB40002000000000000000000000000000000000000000000000000000000000000000000000000000000000000000000000000800600000000000000D8FE58
:3C5AF000020000000000000000000000000000000000000000000000000000000000000000000000000000000000000000000000002000000000008001009EFF3A
:3C5B2C0002000000000000000000000000000000000000000000000000000000000000000000000000000000000000000000000000A406000000009006000AFEF3
:3C5B6800000000000000000000000000000000000000000000000000000000000000000000000000000000000000000000000000000006000000000006001EFED9
:3C5BA4000000000000000000000000000000000000000000000000000000000000000000000000000000000000000000000000000080000000000080060078FE49
:3C5BE00002000000000000000000000000000000000000000000000000000000000000000000000000000000000000000000000000803000000000A006007BFEB8
:3C5C1C0002000000000000000000000000000000000000000000000000000000000000000000000000000000000000000000000000840800000000800000A3FF9C
:3C5C5800020000000000000000000000000000000000000000000000000000000000000000000000000000000000000000000000000002000000000000001CFEF2
:3C5C9400020000000000000000000000000000000000000000000000000000000000000000000000000000000000000000000000008002000000008000000DFFC4
:3C5CD0000A08000000000000000000000000000000000000000000000000000000000000000000000000000000000000000000000040060100000000000091FFAF
:3C5D0C0002900000000000000000000000000000000000000000000000000000000000000000000000000000000000000000000000000000000000D00800E7FF0B
:3C5D48000000000000000000000000000000000000000000000000000000000000000000000000000000000000000000000000000000000000000000060078FEA3
:3C5D840000800600000000000000000000000000000000000000000000000000000000000000000000000000000000000000000000000000000000000000F8FE67
:3C5DC00002A006000000000000000000000000000000000000000000000000000000000000000000000000000000000000000000000000000000008006010EFE6C
:3C5DFC0002800000000000000000000000000000000000000000000000000000000000000000000000000000000000000000000000000000000000221200BFFEF8
:3C5E380002000000000000000000000000000000000000000000000000000000000000000000000000000000000000000000000000000000000000800000AFFFFE
:3C5E740002000600000000000000000000000000000000000000000000000000000000000000000000000000000000000000000000000000000000800000D8FE94
:3C5EB0000200060000000000000000000000000000000000000000000000000000000000000000000000000000000000000000000000000000000000000418FE94
:3C5EEC00008000000000000000000000000000000000000000000000000000000000000000000000000000000000000000000000000000000000008100001FFE5C
:3C5F2800000000000000000000000000000000000000000000000000000000000000000000000000000000000000000000000000000000000000000000001EFE21
:3C5F640000800600000000000000000000000000000000000000000000000000000000000000000000000000000000000000000000000000000000000000F8FE85
:3C5FA00002800000000000000000000000000000000000000000000000000000000000000000000000000000000000000000000000000000000000C00810F6FF76
:3C5FDC0002B00000000000000000000000000000000000000000000000000000000000000000000000000000000000000000000000000000000000000200BDFF19
:3C601800020006000000000000000000000000000000000000000000000000000000000000000000000000000000000000000000000000000000000004000DFF34
:3C60540000000600000000000000000000000000000000000000000000000000000000000000000000000000000000000000000000000000000000800000F8FE94
:3C609000000000000000000000000000000000000000000000800100000000000000000000000000000000000000000000000000000000800100000030000CFF97
:3C60CC0000800000000000000000000000000000000000000000000000000000000000000000000000000000000000000000000040801600000000801000BCFEF8
:3C610800000000000000000000000000000000000000000000000000000000000000000000000000000000000000000000000000000002000000000000003CFE1F
:3C614400008006000000000000000000000000000000000000000000000000000000000000000000000000000000000000000000000000000000008002005AFEBF
:3C61800002800000000000000000000000000000000000000000000000000000000000000000000000000000000000000000000000A02200000000800204CDFF4D
:3C61BC0002D00000000000000000000000000000000000000000000000000000000000000000000000000000000000000000000000220000000000800C0091FF97
:3C61F800000006000000000000000000000000000000000000000000000000000000000000000000000000000000000000000000000000000000000002005AFE0B
:3C6234000200060000000000000000000000000000000000000000000000000000000000000000000000000000000000000000000080000000000080000049FFDE
:3C6270000200000000000000000000000000000000000000000000800100000000000000000000000000000000000000000000000000160200000000000171FEE7
:3C62AC0000800000000000000000000000000000000000000000000000000000000000000000000000000000000000000000000000900E00000000D0160057FE5D
:3C62E800000000000000000000000000000000000000000000000000000000000000000000000000000000000000000000000000000002000000000006005AFE1A
:3C63240000800600000000000000000000000000000000000000000000000000000000000000000000000000000000000000000000800600000000800600F8FEB5
:3C63600002800600000000000000000000000000000000000000000000000000000000000000000000000000000000000000000000C00601000000800604C8FE62
:3C639C0002800600000000000000000000000000000000000000000000000000000000000000000000000000000000000000000000A40800000000800A00CFFF39
:3C63D800020006000000000000000000000000000000000000000000000000000000000000000000000000000000000000000000000000000000000004000DFF71
:3C641400000000000000000000000000000000000000000000000000000000000000000000000000000000000000000001000000008004000000008000005AFFEE
:3C645000000000000000000000000000000000000000000000000000000000000000000000000000000000000000008000000000000000080000000000010EFE7B
:3C648C0000A20000000000000000000000000000000000000000000000000000000000000000000000000000000000000000000000880E000000008006002DFFEA
:3C64C800000006000000000000000000000000000000000000000000000000000000000000000000000000000000000000000000000002000000000006003CFE50
:3C6504000000000000000000000000000000000000000000000000000000000000000000000000000000000000000000000000000080060000000080000078FEDF
:3C65400002800600000000000000000000000000000000000000000000000000000000000000000000000000000000000000000000C00601000000803000FCFF25
:3C657C0002100000000000000000000000000000000000000000000000000000000000000000000000000000000000000000000000A400000000008000001BFF93
:3C65B8000000068000800080008000800080008000800080008000800080008000800080008000800080008000800080008000800080008000800080000069FFB9
:3C65F400020000000000000000000000000000000000000000000000000000000000000000000000000000000000000000000000000004000000000007001CFF43
:3C663000022006000000000000000000008001000000000000000000000000000000000000000000000000000000000000000000000010020000008006002EFEC1
:3C666C00000000000000000000000000000000000000000000000000000000000000000000000000000000000000000000000000000000000000000000001EFED6
:3C66A80000200000000000000000000000000000000000000000000000000000000000000000000000800000000000000000000000200000000000200000BEFE1A
:3C66E400000000000000000000000000000000000000000000000000000000000000000000000000000000000000000000000000000000000000000000001EFE5E
:3C672000000000000000000000000000000000000000000000000000000000000000000000000000000000000000000000000000000000000000000000001EFE21
:3C675C00000000000000000000000000000000000000000000000000000000000000000000000000000000000000000000000000000000000000000000001EFEE5
:3C679800000000000000000000000000000000000000000000000000000000000000000000000000000000000000000000000000002000000000000000200DFF79
:3C67D400000000000000000000000000000000000000000000000000000000000000000000000000000000000000000000000000000000000000000000001EFE6D
:3C681000000000000000000000000000000000000000000000000000000000000000000000000000000000000000000000000000000000000000000000001EFE30
:3C684C000000000000000000000000000000000000000000000000000000000000000000000000000000000000000000000000000004000000002000010038FFB4
:3C688800000200000000000000000000000002000000000000000000000000000000000000000000000000000000000000000000000000000000000000003EFE94
:3C68C400000000000000000000000000000000000000000000000000000000000000000000000000000000000000000000000000000000000000000000001EFE7C
:3C690000000000000000000000000000000000000000000000000000000000000000000000000000000000000000000000000000000000000000000000001EFE3F
:3C693C00000000000000000000000000000000000000000000000000000000000000000000000000000000000000000000000000000000000000000000001EFE03
:3C69780000000000000000000000000000000000000000000000000000000000000000000000000000000000000000000200000008000001000000000101BCFF1B
:3C69B400000000000000000000000000000000000000000000000000000000000000000000000000000000000000000000000000000000000000000000001EFE8B
:3C69F00000000000000000000000000000000000000000000000000000000000000000000000000000000000000000000000000000000002000000000480F2FEF5
:3C6A2C00000000000000000000000000000000000000000000000000000000000000000000000000000000000000000000000000000000000000000000001EFE12
:3C6A6800000000000000000000000000000000000000000000000000000000000000000000000000000000000000000000000000000000000000000000001EFED6
:3C6AA400000000000000000000000000000000000000000000000000000000000000000000000000000000000000000000000000000000000000000000001EFE9A
:3C6AE000000000000000000000000000000000000000000000000000000000000000000000000000000000000000000000000000000000000000000000001EFE5E
:3C6B1C00000000000000000000000000000000000000000000000000000000000000000000000000000000000000000000000000000000000000000000001EFE21
:3C6B5800000000000000000000000000000000000000000000000000000000000000000000000000000000000000000000000000000000000000000000001EFEE5
:3C6B9400000000000000000000000000000000000000000000000000000000000000000000000000000000000000000000000000000000000000000000001EFEA9
:3C6BD000000000000000000000000000000000000000000000000000000000000000000000000000000000000000000000000000000000000000000000001EFE6D
:3C6C0C00000000000000000000000000000000000000000000000000000000000000000000000000000000000000000000000000000000000000008000009EFE30
:3C6C4800000000000000000000000000000000000000000000000000000000000000000000000000000000000000000000000000000000000000000000001EFEF4
:3C6C8400000000000000000000000000000000000000000000000000000000000000000000000000000000000000000000000000000000000000000000001EFEB8
:3C6CC000000000000000000000000000000000000000000000000000000000000000000000000000000000000000000000000000000400002000000400003EFE34
:3C6CFC00000000000000000000000000000000000000000000000000000000000000000000000000000000000000000000000000000000000000000000001EFE40
:3C6D3800000000000000000000000000000000000000000000002000000000000000000000000000000000000000000000000000000000000100000000002EFFD1
:3C6D7400000000000000000000000000000000000000000000000000000000000000000000000000000000000000000000000000000000000000000000001EFEC7
:3C6DB000000000000000000000000000000000000000000000000000000000000000000000000000000000000000000000000000000000000000000000001EFE8B
:3C6DEC00000000000000000000000000000000000000000000000000000000000000000000000000000000000000000000000000000000000000000000001EFE4F
:3C6E28000000000000000000000000000000000000000000000000001000000000000000000000000000000000000000000000000008000000000000000016FF01
:3C6E64000000000000000000000000000000000000000000000000000000000000000000000000000000000000000000000000000028020000000000000014FEB6
:3C6EA000000000000000000000000000000000000000000000000000000000000000000000000000000200000000000000000000000000000000000200001EFE96
:3C6EDC00020000000000000000000000000000000000000000000000000000000000000000000000000000000000000000000000000000000000000000002FFF4A
:3C6F1800000000000000000000000000000000000000000000000000000000000000000000000000000000000000000000000000000000000000000000001EFE21
:3C6F5400000000000000000000000000000000000000000000000000000000000000000000000000000000000000000000000000000000000000000000001EFEE5
:3C6F9000000000000000000000000000000000000000000000000000000000000000000000000000000000000000000000000000000000000000000000001EFEA9
:3C6FCC00000000000000000000000000000000000000000000000000000000000000000000000000000000000000000000000000000000000000000000001EFE6D
:3C700800000000000000000000000000000000000000000000000000000000000000000000000000000000000000000000000000000000000000000000001EFE30
:3C704400000000000000000000000000000000000000000000000000000000000000000000000000000000000000000000000000000000000000000000001EFEF4
:3C708000000000000000000000000000000000000000000000000000000000000000000000000000000000000000000000000000000000000000000000001EFEB8
:3C70BC00000000000000000000000000000000000000000000000000000000000000000000000000000000000000000000000000000000000000000000001EFE7C
:3C70F800000000000000000000000000000000000000000000000000000000000000000000000000000000000000000000000000000000000000000000001EFE40
:3C713400000000000000000000000000000000000000000000000000000000000000000000000000000000000000000000000000000000000000000000001EFE03
:3C717000020000000000000000000000000000000000000000000000000000000000000000000000000000000000000000000000000000000000000000002FFFB3
:3C71AC00020000000000000000000000000000000000000000000000000000000000000000000000000000000000000000000000000000000000000000002FFF77
:3C71E800020000000000000000000000000000000000000000000000000000000000000000000000000000000000000000000000000000000000000000003EFE2D
:3C722400000000000000000000000000000000000000000000000000000000000000000000000000000000000000000000000000000000000000000000000FFF20
:3C726000000000000000000000000000000000000000000000000000000000000000000000000000000000000000000000000000000000000000000000000FFFE4
:3C729C00000000000000000000000000000000000000000000000000000000000000000000000000000000000000000000000000000000000000000000001EFE9A
:3C72D800000000000000000000000000000000000000000000000000000000000000000000000000000000000000000000000000000000000000000000001EFE5E
:3C731400000000000000000000000000000000000000000000000000000000000000000000000000000000000000000000000000000000000000000000001EFE21
:3C735000020000000000000000000000000000000000000000000000000000000000000000000000000000000000000000000000000000000000000000002FFFD1
:3C738C00020000000000000000000000000000000000000000000000000000000000000000000000000000000000000000000000000000000000000000002FFF95
:3C73C800020000000000000000000000000000000000000000000000000000000000000000000000000000000000000000000000000000000000000000003EFE4B
:3C740400000000000000000000000000000000000000000000000000000000000000000000000000000000000000000000000000000000000000000000000FFF3E
:3C744000000000000000000000000000000000000000000000000000000000000000000000000000000000000000000000000000000000000000000000000FFF02
:3C747C0000000000000000000000000000000000000000000000000000000000000000000000000000000000000000000000000000000000000000A40E0054FED0
:3C74B800000000000000000000000000000000000000000000000000000000000000000000000000000000000000000000000000000000000000000000001EFE7C
:3C74F40000000000000000000000000000000000000000000000000000000000000000000000000000000000000000000000000000000000000000800600F8FEE0
:3C75300002000000000000000000000000000000000000000000000000000000000000000000000000000000000000000000000000000000000000800601D9FFBE
:3C756C0002000000000000000000000000000000000000000000000000000000000000000000000000000000000000000000000000000000000000840000ABFFB3
:3C75A800000000000000000000000000000000000000000000000000000000000000000000000000000000000000000000000000000000000000000000001EFE8B
:3C75E40002000000000000000000000000000000000000000000000000000000000000000000000000000000000000000000000000000000000000800000AFFF3B
:3C76200002000000000000000000000000000000000000000000000000000000000000000000000000000000000000000000000000000000000000A00700E9FE9E
:3C765C0000000000000000000000000000000000000000000000000000000000000000000000000000000000000000000000000000000000000000A20E0052FEF2
:3C769800000000000000000000000000000000000000000000000000000000000000000000000000000000000000000000000000000000000000000000001EFE9A
:3C76D40000000000000000000000000000000000000000000000000000000000000000000000000000000000000000000000000000000000000000800600F8FEFE
:3C77100002000000000000000000000000000000000000000000000000000000000000000000000000000000000000000000000000000000000000800601D9FFDC
:3C774C0002000000000000000000000000000000000000000000000000000000000000000000000000000000000000000000000000000000000000C20000EDFF51
:3C778800020000000000000000000000000000000000000000000000000000000000000000000000000000000000000000000000000000000000000000003EFE87
:3C77C400000000000000000000000000000000000000000000000000000000000000000000000000000000000000000000000000000000000000008000008FFF7B
:3C7800000000000000000000000000000000000000000000000000000000000000000000000000000000000000000000000000000000000000000000060069FFDE
:3C783C0000000000000000000000000000000000000000000000000000000000000000000000000000000000000000000000000000000000000000900600E8FE94
:3C7878000000000000000000000000000000000000000000000000000000000000000000000000000000000000000000000000000000000000000000060078FE58
:3C78B40000000000000000000000000000000000000000000000000000000000000000000000000000000000000000000000000000000000000000800400DAFE3C
:3C78F00002000000000000000000000000000000000000000000000000000000000000000000000000000000000000000000000000000000000000A01401CBFEDC
:3C792C000200000000000000000000000000000000000000000000000000000000000000000000000000000000000000000000000000000000000080080027FF6F
:3C796800020000000000000000000000000000000000000000000000000000000000000000000000000000000000000000000000000000000000000000003EFEA5
:3C79A40000000000000000000000000000000000000000000000000000000000000000000000000000000000000000000000000000000000000000800400CBFF59
:3C79E000000000000000000000000000000000000000000000000000000000000000000000000000000000000000000000000000000000000000000002013DFF2C
:3C7A1C0000000000000000000000000000000000000000000000000000000000000000000000000000000000000000000000000000000000000000840E28C7FFAE
:3C7A5800000000000000000000000000000000000000000000000000000000000000000000000000000000000000000000000000000000000000000002003CFEB6
:3C7A940000000000000000000000000000000000000000000000000000000000000000000000000000000000000000000000000000000000000000800200BCFE7A
:3C7AD00002000000000000000000000000000000000000000000000000000000000000000000000000000000000000000000000000000000000000C00210CDFEDB
:3C7B0C00020000000000000000000000000000000000000000000000000000000000000000000000000000000000000000000000000000000000408014083FFE22
:3C7B4800000000000000000000000000000000000000000000000000000000000000000000000000000000000000000000000000000000000000000002002DFFD3
:3C7B840002000000000000000000000000000000000000000000000000000100000000000000000000000100000000000000000000000000000000800400EBFF53
:3C7BC00002000000000000000000000000000000000000000000000000800080010000000000000000800000000000000000000000000000000000200050C2FED6
:3C7BFC0000000000000000000000000000000000000000000000000000000000000000000000000000000000000000000000000000000000000000800E0070FE51
:3C7C38000000000000000000000000000000000000000000000000000000000000000000000000000000000000000000000000000000000000000000060078FE94
:3C7C740000000000000000000000000000000000000000000000000000000000000000000000000000000000000000000000000000000000000000800200BCFE98
:3C7CB000020000000000000000000000000000000000000000000000000000000000000000000000000000000000000000000000000000000000008002108DFE79
:3C7CEC0002000000000000000000000000000000000000000000000000000000000000000000000000000000000000000000000000000000000000800C0063FF6C
:3C7D2800000000000000000000000000000000000000000000000000000000000000000000000000000000000000000000000000000000000000000002003CFEE3
:3C7D640002000000000000000000000000000000000000000000000001000000000000000000000000000000000000000000000000000000000000800700D9FE82
:3C7DA00002000000000000000000000000000000000000000000008000000000000000000000000000000000000000000000000000000000000000800601D1FFCE
:3C7DDC0000000000000000000000000000000000000000000000000000000000000000000000000000000000000000000000000000000000000080800E284BFFEB
:3C7E1800000000000000000000000000000000000000000000000000000000000000000000000000000000000000000000000000000000000000000002003CFEF2
:3C7E540000000000000000000000000000000000000000000000000000000000000000000000000000000000000000000000000000000000000000800200BCFEB6
:3C7E900002000000000000000000000000000000000000000000000000000000000000000000000000000000000000000000000000000000000000A00210ADFE57
:3C7ECC0002000000000000000000000000000000000000000000000000000000000000000000000000000000000000000000000000000000000040800410AFFEF7
:3C7F0800020000000000000000000000000000000000000000000000000000000000000000000000000000000000000000000000000000000000000002000DFF2D
:3C7F440000000000000000000000000000000000000000000000000000000000000000000000000000000000000000000000000000000000000000800400CBFFB3
:3C7F800000000000000000000000000000000000000000000000000000000000000000000000000000000000000000000000000000000000000000200850F2FF5C
:3C7FBC0000000000000000000000000000000000000000000000000000000000000000000000000000000000000000000000000000000000000000820E28C1FF11
:3C7FF800000000000000000000000000000000000000000000000000000000000000000000000000000000000000000000000000000000000000000002003CFE11
:3C80340000000000000000000000000000000000000000000000000000000000000000000000000000000000000000000000000000000000000000800200BCFED4
:3C80700002000000000000000000000000000000000000000000000000000000000000000000000000000000000000000000000000000000000000A00210ADFE75
:3C80AC00020000000000000000000000000000000000000000000000000000000000000000000000000000000000000000000000000000000000408004308DFE17
:3C80E800028000800080008000800080008000800080008000800080008000800080008000800080008000800080008000800080008000800080008002008DFFCC
:3C812400000000000000000000000000000000000000000000000000000000000000000000000000000000000000000000000000000000000000000004004BFFD1
:3C8160000000000000000000000000000000000000000000000000000000000000000000000000000000000000000000000000000000000000000020080836FE7F
:3C819C00000000000000000000000000000000000000000000000000000000000000000000000000000000000000000000000000000000000000000000001EFE8B
:3C81D8000000000000000000000000000000000000000000000001800000000000000000000000000000000000000000000000000000000000000020000026FFA5
:3C821400000000000000000000000000000000000000000000000000000000000000000000000000000000000000000000000000000000000000000000001EFE12
:3C825000000000000000000000000000000000000000000000000000000000000000000000000000000000000000000000000000000000000000000000001EFED6
:3C828C00000000000000000000000000000000000000000000000000000000000000000000000000000000000000000000000000000000000000000000001EFE9A
:3C82C800000000000000000000000000000000000000000000000000000000000000000000000000000000000000000000000000000000000000002002001CFE3E
:3C830400000000000000000000000000000000000000000000000000000000000000000000000000000000000000000000000000000000000000000000001EFE21
:3C834000000000000000000000000000000000000000000000000000000000000000000000000000000000000000000000000000000000000000000000001EFEE5
:3C837C00000000000000000000000000000000000000000000000000000000000000000000000000000000000000000000000000000000000000080001009EFF1F
:3C83B800000000000000000000000000000000000000000000000000000000000000000000000000000000000000000000000000000000000000000000001EFE6D
:3C83F400000000000000000000000000000000000000000000000000000000000000000000000000000000000000000000000000000000000000000404005EFEE9
:3C843000000000000000000000000000000000000000000000000000000000000000000000000000000000000000000000000000000000000000000000001EFEF4
:3C846C00000000000000000000000000000000000000000000000000000000000000000000000000000000000000000000000000000000000000000000001EFEB8
:3C84A800000000000000000000000000000000000000000000000000000000000000000000000000000000000000000000000000000000000000000000001EFE7C
:3C84E400000000000000000000000000000000000000000000000000000000000000000000000000000000000000000000000000000000000000000000001EFE40
:3C852000000000000000000000000000000000000000000000000000000000000000000000000000000000000000000000000000000000000000000000001EFE03
:3C855C00000000000000000000000000000000000000000000000000000000000000000000000000000000000000000000000000000000000000000000001EFEC7
:3C859800000000000000000000000000000000000000000000000000000000000000000000000000000000000000000000000000000000000000004000105EFFFA
:3C85D400000000000000000000000000000000000000000000000000000000000000000000000000000000000000000000000000000000000000000000001EFE4F
:3C861000000000000000000000000000000000000000000000000000000000000000000000000000000000000000000000000000000000000000000000001EFE12
:3C864C00000000000000000000000000000000000000000000000000000000000000000000000000000000000000000000000000000000000000000000001EFED6
:3C868800000000000000000000000000000000000000000000000000000000000000000000000000000000000000000000000000000000000000000000001EFE9A
:3C86C4000000000000000000000000000000000000000000000000000000000000000000000000000000000000000000000000000000000000000020800216FEC4
:3C8700000000000000000000000000000000000000000000000000000000000000000000000000000000400000000000000000000000000000000002000018FEE5
:3C873C00000000000000000000000000000000000000000000000000000000000000000000000000000000000000000000000000000000000000000000001EFEE5
:3C8778000000000000000000000000000000000000000000000000000000000000000000000000000000000000000000000000000000000000000000080186FE38
:3C87B400000000000000000000000000000000000000000000000000000000000000000000000000000000000000000000000000000000000000000000045EFE29
:3C87F000000000000000000000000000000000000000000000000000000000000000000000000000000000000000000000000000000000000000000000001EFE31
:3C882C00000000000000000000000000000000000000000000000000000000000000000000000000000000000000000000000000000000000000000000045EFEB0
:3C886800000000000000000000000000000000000000000000000000000000002000000000000000000000000000000000000000000000000000000000002FFF86
:3C88A400000000000000000000000000000000000000000000000000000000000000000000000000000000000000000000000000000000000000000000001EFE7C
:3C88E000000000000000000000000000000000000000000000000000000000000000000000000000000000000000000000000000000000000000000000001EFE40
:3C891C00000000000000000000000000000000000000000000000000000020000000000000000000000000000000000000000000000000000000080000009CFE5D
:3C895800000000000000000000000000000000000000000000000000100000000000000000000000000000000000000000000000000000000000000A000454FF72
:3C899400000000000000000000000000000000000000000000080000000000000000000000000000000000000000000000000000000000000000000001009EFF01
:3C89D000000000000000000000000000000000000000000000000002000000000000000000000000000000000000000000000000000000000000000006005AFE0B
:3C8A0C0000000000000000000000000000000000000000000000000000000000000000000000000000000000000000000000000000000000000000000028ADFF5A
:3C8A4800000000000000000000000000000000000000000000000000000000000000000000000000000000000000000000000000000000000000000000001EFED6
:3C8A8400000000000000000000000000000000000000000000000000000000000000000000000000000000000000000000000000000000000000000000001EFE9A
:3C8AC000020000000000000000000000000000000000000000000000000000000000000000000000000000000000000000000000000000000000000000002FFF4A
:3C8AFC0002000000000000000000000000000000000000000000000000000000000000000000000000000000000000000000000000000000000000000008AFFF86
:3C8B3800020000000000000000000000000000000000000000000000000000000000000000000000000000000000000000000000000000000000000000002FFFD1
:3C8B7400000000000000000000000000000000000000000000000000000000000000000000000000000000000000000000000000000000000000000000000FFFB7
:3C8BB000000000000000000000000000000000000000000000000000000000000000000000000000000000000000000000000000000000000000000000405AFEF1
:3C8BEC00000000000000000000000000000000000000000000000000000000000000000000000000000000000000000000000000000000000000000000001EFE31
:3C8C2800000000000000000000000000000000000000000000000000000000000000000000000000000000000000000000000000000000000000000000001EFEF4
:3C8C6400000000000000000000000000000000000000000000000000000000000000000000000000000000000000000000000000000000000000000000001EFEB8
:3C8CA000020000000000000000000000000000000000000000000000000000000000000000000000000000000000000000000000000000000000000000002FFF68
:3C8CDC00020000000000000000000000000000000000000000000000000000000000000000000000000000000000000000000000000000000000000000002FFF2C
:3C8D1800000000000000000000000000000000000000000000000000000000000000000000000000000000000000000000000000000000000000000000001EFE03
:3C8D5400020000000000000000000000000000000000000000000000000000000000000000000000000000000000000000000000000000000000000000002FFFB3
:3C8D9000020000000000000000000000000000000000000000000000000000000000000000000000000000000000000000000000000000000000000000002FFF77
:3C8DCC00000000000000000000D006000000000000000000000000000000000000000000000000000000000000000000000000000000000000000000002867FE08
:3C8E08000000000000000000000006000000000000000000000000000000000000000000000000000000000000000000000000000000000000000000000018FE12
:3C8E4400000000000000000000000400000000000000000000000000000000000000000000000000000000000000000000000000000000000000000000001AFED6
:3C8E80000200000000000000008036000000000000000000000000000000000000000000000000000000000000000000000000000000000000000000000091FF6E
:3C8EBC00020000000000000000100E000000000000000000000000000000000000000000000000000000000000000000000000000000000000000000001021FF2A
:3C8EF8000000000000000000000006000000000000000000000000000000000000000000000000000000000000000000000000000000000000000000000009FF30
:3C8F340002000000000000000080060000000000000000000000000000000000000000000000000000000000000000000000000000000000000000000000A1FFD9
:3C8F70000200000000000000004086000000000000000000000000000000000000000000000000000000000000000000000000000000000000000080014038FF05
:3C8FAC00020000000000000000900E0000A10600000000000000000000000000000000000000000000000000000000000000000000000000000000000028DDFF3E
:3C8FE800000000000000000000000600000006000000000000000000000000000000000000000000000000000000000000000000000000000000000000007EFEC5
:3C9024000000000000000000000000000000060000000000000000000000000000000000000000000000000000000000000000000000000000000000000078FE94
:3C906000020000000000000000A020000080160200000000000000000000000000000000000000000000000000000000000000000000000000000000000073FE09
:3C909C00020000000000000000000600000006000000000000000000000000000000000000000000000000000000000000000000000000000000000000500BFE31
:3C90D800020000000000000000000600000006000000000000000000000000000000000000000000000000000000000000000000000000000000000000004FFF00
:3C9114000200000000000000008006000080000000000000000000000000000000000000000000000000000000000000000000000000000000000000000021FFF7
:3C91500002000000000000000000060000000000000000000000000000000000000000000000000000000000000000000000000000000000000000800100B8FFA3
:3C918C000000000000000000008004000080020000000000000000000000000000000000000000000000000000000000000000000000000000000000000030FE73
:3C91C8000000000000000000000004000000020000000000000000000000000000000000000000000000000000000000000000000000000000000000000038FE2F
:3C9204000000000000000000008002000080040000000000000000000000000000000000000000000000000000000000000000000000000000000000000050FEDA
:3C9240000200000000000000008002000080340000000000000000000000000000000000000000000000000000000000000000000000000000000000000073FE49
:3C927C000200000000000000008004000080120000000000000000000000000000000000000000000000000000000000000000000000000000000000000011FE8F
:3C92B8000000000000000000000002000000040000000000000000000000000000000000000000000000000000000000000000000000000000000000000058FE1E
:3C92F40002000000000000000000020000800400000000000000000000000000000000000000000000000000000000000000000000000000000000000000E9FFCE
:3C933000020000000000000000003400000022000000000000000000000000000000000000000000000000000000000000000000000000000000000000003BFF6F
:3C936C0002000000000000000080000000000000000000000000000000000000000000000000000000000000000000000000000000000000000000000000B6FE8F
:3C93A800000000000000000000000000000000000000000000000000000000000000000000000000000000000000000000000000000000000000000000001EFE6D
:3C93E4000000000000000000008006000000000000000000000000000000000000000000000000000000000000000000000000000000000000000000000090FE39
:3C94200002000000000000000080000000000000000000000000000000000000000000000000000000000000000000000000000000000000000000000000A7FFE8
:3C945C0002000000000000000090000000000000000000000000000000000000000000000000000000000000000000000000000000000000000000000000A7FE9D
:3C9498000200000000000000000006000000000000000000000000000000000000000000000000000000000000000000000000000000000000000000000038FE5A
:3C94D4000200000000000000000006000000000000000000000000000000000000000000000000000000000000000000000000000000000000000000000029FF2C
:3C951000020000000000000000200000000000000000000000000000000000000000000000000000000000000000000000000000000000000000000000000DFFF1
:3C954C0000000000000000000080000000000000000000000000000000000000000000000000000000000000000000000000000000000000000000C8060038FE5F
:3C958800000000000000000000000000000000000000000000000000000000000000000000000000000000000000000000000000000000000000000002003CFE6B
:3C95C4000000000000000000008006000000000000000000000000000000000000000000000000000000000000000000000000000000000000000080020032FE33
:3C9600000200000000000000008000000000000000000000000000000000000000000000000000000000000000000000000000000000000000000080120895FE7F
:3C963C00020000000000000000B000000000000000000000000000000000000000000000000000000000000000000000000000000000000000004080140015FF58
:3C967800000000000000000000000600000000000000000000000000000000000000000000000000000000000000000000000000000000000000000002003AFE76
:3C96B40002000000000000000000060000000000010001000100000000000000000000000000000000000000000000000000000000000000000000800400EDFFFF
:3C96F0000200000000000000000000000000008000800080000000000000008001000000000000000000000000000000000000000000000000000020001097FF75
:3C972C0000000000000000000080000000000000000000000000000000000000000000000000000000000000000000000000000000000000000080800600F8FE85
:3C976800000000000000000000000000000000000000000000000000000000000000000000000000000000000000000000000000000000000000000002003CFE89
:3C97A4000000000000000000008006000000000000000000000000000000000000000000000000000000000000000000000000000000000000000080020032FE51
:3C97E00002000000000000000080000000000000000000000000000000000000000000000000000000000000000000000000000000000000000000A01208B5FE5E
:3C981C00020000000000000000D0000000000000000000000000000000000000000000000000000000000000000000000000000000000000000040800C00EBFE89
:3C985800000000000000000000000600000000000000000000000000000000000000000000000000000000000000000000000000000000000000000002003AFE94
:3C98940002000000000000000000060000000000000001000000000000000000000000000000000000000000000000000000000000000000000000800400FDFF0F
:3C98D0000200000000000000000000000000000000800000000000000000000000000000000000000000000000000000000000000000000000000020001007FEA5
:3C990C0000000000000000000080000000000000000000000000000000000000000000000000000000000000000000000000000000000000000000840628C7FF27
:3C994800000000000000000000000000000000000000000000000000000000000000000000000000000000000000000000000000000000000000000002003CFEA7
:3C9984000000000000000000008006000000000000000000000000000000000000000000000000000000000000000000000000000000000000000080020032FE6F
:3C99C00002000000000000000080060000000000000000000000000000000000000000000000000000000000000000000000000000000000000000C01208D3FE38
:3C99FC000200000000000000008006000000000000000000000000000000000000000000000000000000000000000000000000000000000000004080043003FEB2
:3C9A3800000000000000000000000600000000000000000000000000000000000000000000000000000000000000000000000000000000000000000002002BFFC0
:3C9A740002000000000000000000000000000000000000000000000000000000000000000000000000000000000000000000000000000000000000800400EBFF46
:3C9AB0000200000000000000000000000000000000000000000000000000000000000000000000000000000000000000000000000000000000000020081096FFAB
:3C9AEC0000000000000000000000000000880600000000000000000000000000000000000000000000000000000000000000000000000000000000A4060032FED6
:3C9B28000000000000000000000000000000040000000000000000000000000000000000000000000000000000000000000000000000000000000000020078FE85
:3C9B6400000000000000000000000000008006000000000000000000000000000000000000000000000000000000000000000000000000000000008002005AFE65
:3C9BA00002000000000000000000000000C03600000000000000000000000000000000000000000000000000000000000000000000000000000000801208A9FF4F
:3C9BDC0002000000000000000000100000A100000000000000000000000000000000000000000000000000000000000000000000000000000000408004000FFEC9
:3C9C18000080008000800080000000800080008000800080008000800080008000800080008000800080008000800080008000800080008000800080020034FE5C
:3C9C5400020000000000000000000000000004000000000000000000000000000000000000000000000000000000000000000000000000000000000004002FFF9C
:3C9C90000200000000000000000020000000100200000000000000000000000000000000000000000000000000000000000000000000000000000020080817FE1F
:3C9CCC000000000000000000008000010000000000000000000000000000000000000000000000000000000000000000000000000000000000000000000096FF46
:3C9D080000000000000000000008000000080000000000000000008000000000000000000080008000000080000000000000000000000000000000200000B6FE3B
:3C9D4400000000000000000000000000000000000000000000000000000000000000000000000000000000000000000000000000000000000000000000001EFEC7
:3C9D8000000000000000000000000000000000000000000000000000000000000000000000000000000000000000000000000000000000000000000000001EFE8B
:3C9DBC00000000000000000000000000000000000000000000000000000000000000000000000000000000000000000000000000000000000000000000001EFE4F
:3C9DF8000000000000000000000000000000000000000000000000000000000000000000000000000000000000000000000000000000000000000000008096FE1B
:3C9E3400000000000000000000000000000000000000000000000000000000000000000000000000000000000000000000000000000000000000000000001EFED6
:3C9E7000000000000000000000000000000000000000000000000000000000000000000000000000000000000000000000000000000000000000000000001EFE9A
:3C9EAC0000000000000000000000000000000000000000000000000400000000000000000004000400000000000000000000000000000000000008000100DEFF88
:3C9EE800000000000000000000000000000000000000000000000000000000000000000000000000000000000000000000000000000000000000000000000FFF30
:3C9F2400000000000000000000000000000000000000000000000000000000000000000000000000000000000000000000000000000000000000000000001EFEE5
:3C9F6000000000000000000000000000000000000000000000000000000000000000000000000000000000000000000000000000000000000000000000001EFEA9
:3C9F9C00000000000000000000000000000000000000000000000000000000000000000000000000000000000000000000000000000000000000000000001EFE6D
:3C9FD80000000000000000000080200000000000000000000000000000000000000000000000000000000000000000000000000000000000000000000000B6FEF9
:3CA01400000000000000000000000000000000000000000000000000000000000000000000000000000000000000000000000000000000000000000000001EFEF4
:3CA05000000000000000000000000100000000020000000000000000000000000000000000000000000000000000000000000000000000000000000000003FFE94
:3CA08C00000000000000000000000000000000000000000000000000000000000000000000000000000000000000000000000000000000000000000000001EFE7C
:3CA0C800000000000000000000000000000000000000000000000000000000000000000000000000000000000000000000000000000000000000000000001EFE40
:3CA10400000000000000000000000000000000000000000000000000000000000000000000000000000000000000000000000000000000000000000000001EFE03
:3CA14000000000000000000000000000000000000000000000000000000000000000000000000000000000000000000000000000000000000000000000001EFEC7
:3CA17C00000000000000000000000000000000000000000000000000000000000000000000000000000000000000000000000000000000000000004000401AFE0F
:3CA1B800000000000000000000000000000000000000000000000000000000000000000000000000000000000000000000000000000000000000000000001EFE4F
:3CA1F400000000000000000000000000000000000000000000000000000000000000000000000000000000000000000000000000000000000000000000001EFE13
:3CA23000000000000000000000000000000000000000000000000000000000000000000000000000000000000000000000000000000000000000000000001EFED6
:3CA26C00000000000000000000000000000000000000000000000000000000000000000000000000000000000000000000000000000000000000000000001EFE9A
:3CA2A800000000000000000000000000000000000000000000000000000000000000000000000000000000000000000000000000000000000000000000001EFE5E
:3CA2E400000000000000000000000000000000000000000000000000000000000000000000000000000000000000000000000000000000000000000000045EFEDE
:3CA32000000000000000000000000000000000000000000000000000000000000000000000000000000000000000000000000000000000000000000000001EFEE5
:3CA35C00000000000000000000000000000000000000000000000000000000000000000000000000000000000000000000000000000000000000000000001EFEA9
:3CA39800000000000000000000000000000000000000200000000000000000002000000000000000000000000000000000000000000000000000000001000DFE3D
:3CA3D400000000000000000000000000000000000000000000000000000000000000000000000000000000000000000000000000000000000000000000001EFE31
:3CA41000000000000000000000000000000000000000000000000000000000000000000000000000000000000000000000000000000000000000000000001EFEF4
:3CA44C00000000000000000000000000000000002000000020000000000000000000000000000000000000000000000000000000000000000000082000009CFED2
:3CA488000000000000000000000008008000000000001000000000000000000000000000000000000000000000000000000000000000000000000008000096FF63
:3CA4C400000000000000000000000000000000000000000000000000000000000000000000000000000000000000000000000000000000000000000000001EFE40
:3CA50000000000000000000000000000000200000000000000000000000000000000000000000000000000020000000000000000000000000000000000003CFEE1
:3CA53C0000000000000000000000000000000000000000000000000000000000000000000000000000000000000000000000000000000000000000000048CBFFD1
:3CA57800000000000000000000000000000000000000000000000000000000000000000000000000000000000000000000000000000000000000000000001EFE8B
:3CA5B400000000000000000000000000000000000000000000000000000000000000000000000000000000000000000000000000000000000000000000001EFE4F
:3CA5F000020000000000000000000000000000000000000000000000000000000000000000000000000000000000000000000000000000000000000000002FFFFF
:3CA62C00020000000000000000000000000000000000000000000000000000000000000000000000000000000000000000000000000000000000000000102FFEB3
:3CA66800000000000000000000000000000000000000000000000000000000000000000000000000000000000000000000000000000000000000000000000FFFA8
:3CA6A400020000000000000000000000000000000000000000000000000000000000000000000000000000000000000000000000000000000000000000002FFF4A
:3CA6E000020000000000000000000000000000000000000000000000000000000000000000000000000000000000000000000000000000000000000000407AFE84
:3CA71C000000000000000000000000000000000000000000000000000000000000000000000000000000000000000000000000000000000000008080060070FE8D
:3CA75800000000000000000000000000000000000000000000000000000000000000000000000000000000000000000000000000000000000000000000001EFEA9
:3CA7940000000000000000000000000000000000000000000000000000000000000000000000000000000000000000000000000000000000000000800200BCFE4D
:3CA7D00002000000000000000000000000000000000000000000000000000000000000000000000000000000000000000000000000000000000000C05200D9FE62
:3CA80C0002000000000000000000000000000000000000000000000000000000000000000000000000000000000000000000000000000000000000A40400CFFF98
:3CA84800000000000000000000000000000000000000000000000000000000000000000000000000000000000000000000000000000000000000000002003CFE98
:3CA8840002000000000000000000000000000000000000000000000000000000000000000000000000000000000000000000000000000000000000800400EBFF28
:3CA8C00002000000000000000000000000000000000000000000000000000000000000000000000000000000000000000000000000000000000000002A0087FFAA
:3CA8FC000000000000000000000000000000000000000000000000000000000000000000000000000000000000000000000000000000000000008080060070FEAC
:3CA93800000000000000000000000000000000000000000000000000000000000000000000000000000000000000000000000000000000000000000000001EFEC7
:3CA9740000000000000000000000000000000000000000000000000000000000000000000000000000000000000000000000000000000000000000800200BCFE6B
:3CA9B00002000000000000000000000000000000000000000000000000000000000000000000000000000000000000000000000000000000000000C05200D9FE80
:3CA9EC0002000000000000000000000000000000000000000000000000000000000000000000000000000000000000000000000000000000000000880C006BFF2F
:3CAA2800000000000000000000000000000000000000000000000000000000000000000000000000000000000000000000000000000000000000000002003CFEB6
:3CAA640002000000000000000000000000000000000000000000000000000000000000000000000000000000000000000000000000000000000000800400EBFF46
:3CAAA00002000000000000000000000000000000000000000000000000000000000000000000000000000000000000000000000000000000000000A02300AFFE08
:3CAADC00000000000000000000000000000000000000000000000000000000000000000000000000000000000000000000000000000000A206008080064829FF20
:3CAB1800000000000000000000000000000000000000000000000000000000000000000000000000000000000000000000000000000000000200000000001CFEE5
:3CAB540000000000000000000000000000000000000000000000000000000000000000000000000000000000000000000000000000000000000000800200BCFE89
:3CAB9000020000000000000000000000000000000000000000000000000000000000000000000000000000000000000000000000000000800A0100C052005BFF90
:3CABCC0002000000000000000000000000000000000000000000000000000000000000000000000000000000000000000000000000000010000000821430DBFE9C
:3CAC0800000000000000000000000000000000000000000000000000000000000000000000000000000000000000000000000000000000000000000002002DFFE2
:3CAC44000200000000000000000000000000000000000000000000000000000000000000000000000000000000000000000000000000008000000080050063FE6C
:3CAC8000020000000000000000000000000000000000000000000000000000000000000000000000000000000000000000000000000000408E0000C0220014FED4
:3CACBC0002000000000000000000000000000000000000000000000000000000000000000000000000000000000000000000000000004080160080800600CAFEB6
:3CACF800000000000000000000000000000000000000000000000000000000000000000000000000000000000000000000000000000000000000000000001EFE04
:3CAD34000000000000000000000000000000000000000000000000000000000000000000000000000000000000000000000000000000008002000080020036FEAB
:3CAD7000000000000000000000000000000000000000000000000000000000000000000000000000000000000000000000000000000000A0820000C05200D1FEA4
:3CADAC00020000000000000000000000000000000000000000000000000000000000000000000000000000000000000000000000000000C20400808004008BFF15
:3CADE800020000000000000000000000000000000000000000000000000000000000000000000000000000000000000000000000000000000200000002001EFE0D
:3CAE24000000000000000000000000000000000000000000000000000000000000000000000000000000000000000000000000000000008004000080040047FFA4
:3CAE6000000000000000000000000000000000000000000000000000000000000000000000000000000000000000000000000000000000003200002032002DFE07
:3CAE9C000200000000000000000000000000000000000000000000000000000000000000000000000000000000000000000000000000000000008080064885FFA6
:3CAED800000000000000000000000000000000000000000000000000000000000000000000000000000000000000000000000000000000000000000000001EFE22
:3CAF140000000000000000000000000000000000000000000000000000000000000000000000000000000000000000000000000000000000000000800200BCFEC5
:3CAF500000000000000000000000000000000000000000000000000000000000000000000000000000000000000000000000000000000000000000C05200F9FEBC
:3CAF8C0002000000000000000000000000000000000000000000000000000000000000000000000000000000000000000000000000000000000000842400EDFFF3
:3CAFC800020000000000000000000000000000000000000000000000000000000000000000000000000000000000000000000000000000000000000002000DFF3D
:3CB0040000000000000000000000000000000000000000000000000000000000000000000000000000000000000000000000000000000000000000800500CBFEC2
:3CB0400000000000000000000000000000000000000000000000000000000000000000000000000000000000000000000000000000000000000000C01230CEFE06
:3CB07C00020000000000000000000000000000000000000000000000000000000000000000000000000000000000000000000000000000840600808006484BFF74
:3CB0B800000000000000000000000000000000000000000000000000000000000000000000000000000000000000000000000000000000000200000000001CFE40
:3CB0F40000000000000000000000000000000000000000000000000000000000000000000000000000000000000000000000000000000000000000800200BCFEE4
:3CB13000000000000000000000000000000000000000000000000000000000000000000000000000000000000000000000000000000000A0520000C0520001FEE0
:3CB16C0002000000000000000000000000000000000000000000000000000000000000000000000000000000000000000000000000000010000000821410F9FEF8
:3CB1A800020000000000000000000000000000000000000000000000000000000000000000000000000000000000000000000000000000000000000002000DFF5B
:3CB1E4000000000000000000000000000000000001000100010000000000010000000000000000000000010000000000000000000000008000000080040043FFE4
:3CB22000000000000000000000000000000000800080008000000000008000000000000000000000008000000000000000000000000000408E0000200230F4FF5F
:3CB25C0000000000000000000000000000000000000000000000000000000000000000000000000000000000000000000000000000000090060000C10648F3FF1F
:3CB29800000000000000000000000000000000000000000000000000000000000000000000000000000000000000000000000000000000000600000006007EFEF2
:3CB2D4000000000000000000000000000000000000000000000000000000000000000000000000000000000000000000000000000000008006000080060076FEBE
:3CB31000020000000000000000000000000000000000000000000000000000000000000000000000000000000000000000000000000000C006000080060003FFB1
:3CB34C000200000000000000000000000000000000000000000000000000000000000000000000000000000000000000000000000000008000000080200025FF7F
:3CB38800000000000000000000000000000000000000000000000000000000000000000000000000000000000000000000000000000000000000000000000FFF7B
:3CB3C4000200000000000000000000000000000000000100000001000100000000000000000000000000000000000000000000000000008000000080010037FF11
:3CB400000200000000000000000000000000000000800000008000800000000000000000000000000000000000000000000000000000000000000080004072FE5E
:3CB43C0002000000000000000000000000000000000000000000000000004080060000000000000000000000000000000000000000000080160000C206485BFF0C
:3CB47800000000000000000000000000000000000000000000000000000000000600000000000000000000000000000000000000000000000600000002003CFE50
:3CB4B4000000000000000000000000000000000000000000000000000000000006000000000000000000000000000000000000000000008000000080020032FE24
:3CB4F000000000000000000000000000000000000000000000000000000000A00600000000000000000000000000000000000000000000808000008052001DFE8D
:3CB52C0002000000000000000000000000000000000000000000000000000000000000000000000000000000000000000000000000000080000000D0244075FFB9
:3CB56800020000000000000000000000000000000000000000000000000000000000000000000000000000000000000000000000000000000000000002000DFF97
:3CB5A40000000000000000000000000000000000000000000000000000000080000000000000000000000000000000000000000000000080060000800400CDFF15
:3CB5E0000000000000000000000000000000000000000000000000000000000000000000000000000000000000000000000000000000000006000000081090FF82
:3CB61C0000000000000000000000000000000000000000000000000000000000000000000000000000000000000000000000000000000000000080800248E1FFC8
:3CB65800000000000000000000000000000000000000000000000000000000000000000000000000000000000000000000000000000000000000000002003CFE7A
:3CB6940000000000000000000000000000000000000000000000000000000000000000000000000000000000000000000000000000000000000000800600F8FEFE
:3CB6D00002000000000000000000000000000000000000000000000000000000000000000000000000000000000000000000000000000000000000C05000FBFE33
:3CB70C000200000000000000000000000000000000000000000000000000000000000000000000000000000000000000000000000000000000000088302097FE92
:3CB7480000800080008000800080008000800080008000800080008000800080008000800080008000800080008000800080008000800080008000800600E9FFD7
:3CB78400020000000000000000000000000000000000000000000000000000000000000000000000000000000000000000000000000000000000000000002FFF59
:3CB7C00002000000000000000000000000000000000000000000000000000000000000000000000000000000000000000000000000000000000000C0870090FF75
:3CB7FC00000000000000000000000000000000000000000000000400000000000000000000000000000000000000000000000000000000000000000000001AFEF5
:3CB838000000000000000000000000000000000000000000000000800080000004800000008000000000008000000000000000000000002000000020000098FE7A
:3CB87400000000000000000000000000000000000000000000000000000000000000000000000000000000000000000000000000000000000000000000001EFE7C
:3CB8B000000000000000000000000000000000000000000000000000000000000000000000000000000000000000000000000000000000000000000000001EFE40
:3CB8EC00000000000000000000000000000000000000000000000000000000000000000000000000000000000000000000000000000000000000000000001EFE04
:3CB928000000000000000000000000000000000000000000000000000000000000000000000000000000000000000000000000000000000000000000008096FECF
:3CB96400000000000000000000000000000000000000000000000000000000000400000000000000000000000000000000000000000000000000000000001AFE8B
:3CB9A000000000000000000000000000000000000000000000000000000000000000000000000000000000000000000000000000000000000000000000001EFE4F
:3CB9DC00000000000000000000000000000000000000000000000000000000000000000000000000000000000000000000000000000000002000000001003EFFD1
:3CBA180000000000000000000000000000000000000000000000000000000000000000000000000000000000000000000000000000000082000000000000A7FFCA
:3CBA5400000000000000000000000000000000000000000000000000000000000000000000000000000000000000000000000000000000000000000000001EFE9A
:3CBA9000000000000000000000000000000000000000000000000000000000000000000000000000000000000000000000000000000000000000000000001EFE5E
:3CBACC00000000000000000000000000000000000000000000000000000000000000000000000000000000000000000000000000000000000000000000001EFE22
:3CBB080002000000000000000000000000000000000000000000000000000800000000000000000000000000000000000000000000000000000000000000B6FE43
:3CBB4400000000000000000000000000000000000000000000000000000000000000000000000000000000000000000000000000000000001000400004000EFE65
:3CBB8000000000000000000000000000000000000000000000000000000000000000000000000000000000000000000000000000000000000000000000001EFE6D
:3CBBBC00000000000000000000000000000000000000000000000000000000000000000000000000000000000000000000000000000000000000000000001EFE31
:3CBBF80000000000000000000000000000000000000000000000000000000000000000000000000000000000000000000000000000000040000000000018DAFFE0
:3CBC3400000000000000000000000000000000000000000000000000000000000000000000000000000000000000000000000000000000000000000000001EFEB8
:3CBC7000000000000000000000000000000000000000000000000002000000000000000000020000000000020000000000000000000000000000000000003CFE58
:3CBCAC00000000000000000000000000000000000000000000001000000000000000000000000000000000000000000000000000000000020000000200002CFE1E
:3CBCE800000000000000000000000000000000000000000000000000000000000000000000000000000000000000000000000000000000000000000000001EFE04
:3CBD2400000000000000000000000000000000000000000000000000000000000000000000000000000000000000000000000000000000200000000000003CFE89
:3CBD60000000000000000000000000000000000000000000000000000000000000000000000000000000400000000000000000000000000000000002000018FE4F
:3CBD9C00000000000000000000000000000000000000000000000000000000000000000000000000000000000000000000000000000010000000004010005EFEAF
:3CBDD800000000000000000000000000000000000000000000000000000000000000000000000000000000000000000000000000000000400000000100004AFFA5
:3CBE1400000000000000000000000000000000000000000000000000000000000000000000000000000000000000000000000000000000000000000000045EFE92
:3CBE50000000000000000000000000000000000020000000000000000000000000000000000000000000000000000000000000000000000000000008000036FE5A
:3CBE8C000000000000000000000000000000000000000000000000000000001000000000000000000000000000000000000000000000000008000100818086FEDC
:3CBEC80000000000000000000000000000000000000020000000000000000000000000000000000000000000000000000000000000000000000000000840F0FEE8
:3CBF0400000000000000000000000000000000000000000000000000000000000000000000000000000000000000000000000000000000000000000000001EFEE5
:3CBF400000000000000000000000000000000000000008000000000000000000000000000000000000000000000000000000000000000000000000200000BEFEE1
:3CBF7C0000000000000000000000000000000000000000002000000000002000000000000000000000000000000000000000000000000000000008200000BEFE65
:3CBFB8000000000000000000000000000000000000000000000000001000000000000000000000000000000000000000000000000000000020000008100026FEE1
:3CBFF40000000000000000000000000000000000000000000000020000000008000000000000000000000000000000000000000000000008040000200008B8FE1D
:3CC03000000000000000000000000000000000000000000000000000000200000002000000000000000000000000000000000000000000000000000000425AFE36
:3CC06C0000000000000000000000000000000000000000000000000000000000000000000000000000000000000000000000000000000000004800480000DAFE30
:3CC0A80000000000000000000000000000000000000000000000000000000000000000000000000000000000000000000400000000000000008000800000D2FE88
:3CC0E40000000400040004800000008000800480040000000480040000000000000000000000048004800000048004000480040000000000008000800000D6FE98
:3CC12000000000800080000004800400040000000080048000000080048004800480048004800000000004800000008000000080048004800480048000005EFE4F
:3CC15C000000048004800480048004800480048004800480048004800480048004800480048004800480048004800480048004800480048024800488000036FE5F
:3CC1980000000400040004800000008000800480040000000480040000000000000000000000048004800000048004000480040000000000008000800000D6FEE3
:3CC1D400000000800080000004800400040000000080048000000080048004800480048004800000000004800000008000000080048004800480048000005EFE9B
:3CC210000000008000800000048004000400000000800480000000800480048004800480048000000000048000000080000000800480048004200440000094FEC8
:02C24C00FFFFF2
:00000001FF
